:020000040800F2
:10000000D85F00209D0100089954000801460008AF
:1000100011530008C90F0008255E00080000000009
:100020000000000000000000000000004157000830
:10003000F117000800000000D156000875570008AD
:10004000B7010008B7010008B7010008B7010008B0
:10005000B7010008B7010008F5170008B70100084C
:10006000B7010008B7010008FD170008B701000834
:1000700069150008B7010008B7010008B7010008BA
:10008000B7010008B7010008B7010008E50F000834
:10009000CD0F0008D90F0008B701000805180008A7
:1000A000B7010008B7010008B7010008B701000850
:1000B000B7010008B7010008B7010008B701000840
:1000C000B7010008B7010008B7010008B701000830
:1000D000B7010008255D0008B7010008315D000880
:1000E000B7010008B7010008B7010008B701000810
:1000F000B7010008B7010008B7010008B701000800
:10010000B7010008B7010008B7010008B7010008EF
:10011000B7010008B7010008B701000849580008F6
:10012000B701000875150008811500088D15000835
:10013000B7010008B7010008B7010008B7010008BF
:10014000F10F0008FD0F0008B7010008B701000813
:1001500099150008A5150008B7010008095E0008F8
:10016000B7010008B7010008B7010008B70100088F
:10017000B7010008B7010008B7010008000000003F
:10018000B7010008B7010008DFF80CD000F056FAFC
:1001900000480047C15E0008D85F0020064880473D
:1001A00006480047FEE7FEE7FEE7FEE7FEE7FEE75C
:1001B000FEE7FEE7FEE7FEE7355800088901000884
:1001C0002DE9F05F0546002092469B46884606468C
:1001D000814640241BE0284641464746224600F01F
:1001E0006DF953465A46C01A914110D3114618462C
:1001F000224600F054F92D1A67EB01084F462246BB
:100200000120002100F04BF917EB00094E41201EA0
:10021000A4F10104DFDC484631462A464346BDE8E6
:10022000F09F00000649074A0868504343F239022C
:10023000104408604008704701490860704700009A
:10024000000000206D4EC64140EA01039B0703D029
:1002500009E008C9121F08C0042AFAD203E011F805
:10026000013B00F8013B521EF9D27047D2B201E0C7
:1002700000F8012B491EFBD270470022F6E710B5AB
:1002800013460A4604461946FFF7F0FF204610BD04
:100290002DE9F04D81EA030404F0004B21F0004504
:1002A00014464FF0000A23F0004150EA050220D026
:1002B00054EA01021DD0C5F30A570246C5F31303E1
:1002C000C1F31300C1F30A5640F4801543F48013C0
:1002D000A7EB0608101BD64608F2FD3873EB0500A5
:1002E00002D308F1010801E092185B41B8F1000F58
:1002F00003DA00200146BDE8F08D00204FF48011A4
:10030000064684460EE0171B73EB050705D3121B48
:1003100063EB050306434CEA010C49084FEA300041
:1003200092185B4150EA0107EDD152EA030012D066
:1003300082EA040083EA0501084305D0101BAB41A3
:1003400006D20122002306E000224FF0004302E023
:100350006FF0010253101AEB06004CEB085110EB42
:100360000A0041EB0B01BDE8F04D00F0EEB830B5EE
:10037000041E71F1000404DB4FF00044404264EBC2
:100380000101141E73F1000405DB1C464FF000430D
:10039000524263EB0403801A994101D3012030BD1E
:1003A000002030BD30B5041E71F1000404DB4FF0B5
:1003B0000044404264EB0101141E73F1000405DBAC
:1003C0001C464FF00043524263EB0403101A8B416A
:1003D00001D3012030BD002030BD30B5041E71F1C5
:1003E000000404DB4FF00044404264EB0101141EA2
:1003F00073F1000405DB1C464FF00043524263EBEF
:100400000403801A994101D2012030BD002030BD83
:1004100030B4044696230800214604D0B62330BCED
:10042000002200F064B820460021F8E70EB540F243
:10043000334102910021CDE900110A460B4600F03C
:1004400093F803B000BDC1F30A5210B5C1F3130114
:1004500040F2FF3341F480119A4201DA002010BDCE
:1004600040F233439A42A2F2334203DC524200F09C
:1004700025F810BD904010BD00F0004230F0004063
:100480000AD0C10D01F56071C0F3160042EA0151B6
:10049000C208400711437047002001467047202AD8
:1004A00004DB203A00FA02F1002070479140C2F1CB
:1004B000200320FA03F3194390407047202A04DBFD
:1004C000203A21FA02F00021704721FA02F3D040CD
:1004D000C2F1200291400843194670470029A8BF85
:1004E0007047401C490008BF20F00100704710B45D
:1004F000B0FA80FC00FA0CF050EA010404BF10BC12
:10050000704749B1CCF1200421FA04F411FA0CF13E
:1005100018BF012121430843A3EB0C01CB1D4FEA77
:1005200000614FEA102042BF002010BC704700EB72
:10053000C35010440029A4BF10BC7047401C4900A0
:1005400008BF20F0010010BC704710B5141E73F1F5
:10055000000408DA401C41F1000192185B411A4383
:1005600001D120F0010010BD2DE9F04D92469B46CF
:1005700011B1B1FA81F202E0B0FA80F22032904675
:10058000FFF78DFF04460F4640EA0A0041EA0B01DF
:1005900053465A46084313D0114653EA010019D076
:1005A000C8F140025046FFF789FF05460E46504607
:1005B00059464246FFF773FF084305D0012004E087
:1005C00020463946BDE8F08D0020054346EAE07636
:1005D0002C4337430A986305E40AA0EB0800002285
:1005E000FD0A44EA47540A3002D500200146E9E7F3
:1005F000010510196941DDE9084500196941BDE8A7
:10060000F04DA2E7002801DBC0F10040002901DB2A
:10061000C1F10041814202D24FF0004004E04FF0AE
:10062000005001D14FF0C040EFF3008121F07F4135
:1006300041EA000181F3008870470000064C074D35
:1006400006E0E06840F0010394E8070098471034A2
:10065000AC42F6D3FFF79CFDD4940008F494000854
:10066000B4EEE00AB1EE602AB0EE401AF1EE10FAF4
:10067000B4EEC02AC8BFB0EE601AF1EE10FAC8BFDF
:10068000B0EE421AB0EE410A704700007047000019
:100690002DE9F04140F250240746984615460E4693
:1006A000C2F20004207801281EBFFD2040B2BDE840
:1006B000F08175B3A068642105F0A0FD00281EBF7D
:1006C000FB2040B2BDE8F081E06818B91AE000BF35
:1006D0000069B8B10178B94204BF4168B142F7D1AD
:1006E0008668A06805F0F4FD7EB1304629460022F8
:1006F000434605F0BDFC002818BF4FF0FF3040B264
:10070000BDE8F081A06805F0E3FDFC2040B2BDE843
:10071000F081FE2040B2BDE8F0810000F0B58BB062
:1007200040F25025C2F20005287808B1FD2075E09E
:1007300005F110006821FFF7A0FD41F2CC00002474
:10074000C2F20000C0F80044C0F80444C0F80848F1
:10075000C0F80C4840F28D60C0F6000068600020D0
:1007600005F076FD0028A86057D001260E270794D3
:1007700001A92E70CDE90544CDE90344CDE901443A
:10078000CDE90344CDE908660A97059440F62C1498
:10079000C2F20004204601F099F8204601F0E8FC7E
:1007A000287801280BD140F6DD00C0F60000A862D1
:1007B00040F6F950C0F60000C5E90400A86140F613
:1007C0002C100321C2F2000001F024F840F654146A
:1007D00001A9CDE90567C2F20004204601F076F8D0
:1007E000204601F0C5FC287801280BD140F6B12045
:1007F000C0F60000686640F6F950C0F60000C5E992
:100800001100E86440F654101121C2F2000001F01A
:1008100001F801202870002000E0FF2040B20BB05A
:10082000F0BD00002DE9F04140F250270646144685
:100830000D46C2F20007387801281EBFFD2040B2E5
:10084000BDE8F081B868642105F0D8FC002C08BF31
:100850000A2400281EBFFB2040B2BDE8F081F868E2
:1008600010B908E0006930B10178B14204BF4168B5
:10087000A942F7D12BE0142000F042FB8046B8F1EA
:10088000000F1AD020461C21002205F031FC002860
:10089000C8F8080018D088F80060C8F8045088F834
:1008A0000C40F868C8F81000C7F80C80B86805F06C
:1008B0000FFD002040B2BDE8F081B86805F008FDEA
:1008C000FE2040B2BDE8F081404600F017FBB8685A
:1008D00005F0FEFCFF2040B2BDE8F0812DE9F04FAD
:1008E00091B040F62C1000214FF0000BC2F2000036
:1008F00001F07AF801A9002801F10D01009165D0FD
:1009000040F62C1540F250280AAE08AFC2F200059E
:10091000C2F200082846002132463B4601F078F832
:1009200000284DD1DDE90C0132464FF002090028C4
:1009300018BF04320428A0F10400146808BF4FF067
:100940000309B0FA80F0022918BF4FEA5019D8F80D
:10095000042020461AB15FFA89F120469047D8F862
:100960000C1019B92CE000BF096949B30A78002AB4
:10097000FAD14A688242F7D1D1F808A0BAF1000F43
:100980001ED0CDF81CB0CDE905BBCDE903BBCDE948
:1009900001BB8DF80490CDE902400D980E9A002815
:1009A0008DF8102003D100983946FFF74DFC02F076
:1009B000C9F80790504601A90022002305F0D8FB92
:1009C0002846002101F010F80028A3D140F6541069
:1009D00000214FF0000BC2F2000001F005F80028E2
:1009E00062D040F6541540F250280AAE0DF12009AD
:1009F000C2F20005C2F200082846002132464B46EA
:100A000001F006F8002849D1DDE90C013246022741
:100A1000002818BF04320428A0F10400146808BF9D
:100A20000327B0FA80F0022918BF4709D8F804203C
:100A3000204612B1F9B220469047D8F80C1019B9E7
:100A40002CE000BF096949B30A78012A04BF4A684B
:100A50008242F7D1D1F808A0BAF1000F1ED0CDF82C
:100A60001CB0CDE905BBCDE903BBCDE901BB8DF8D9
:100A70000470CDE902400D980E9A00288DF81020E0
:100A800003D100984946FFF7DFFB02F05BF80790BF
:100A9000504601A90022002305F06AFB28460021E8
:100AA00000F0A2FF0028A7D111B0BDE8F08F000030
:100AB0002DE9F04F91B040F62C100121C2F2000058
:100AC00000F092FF01A9002801F10D01009165D00D
:100AD00040F62C1540F2502B0AAE0DF120094FF0D4
:100AE0000008C2F20005C2F2000B00BF2846012137
:100AF00032464B4600F08CFF002849D1DDE90C015D
:100B000032460227002818BF04320428A0F104004E
:100B1000146808BF0327B0FA80F0022918BF4709FC
:100B2000DBF80420204612B1F9B220469047DBF8EA
:100B30000C1019B92CE000BF096949B30A78002AE2
:100B4000FAD14A688242F7D1D1F808A0BAF1000F71
:100B50001ED0CDF81C80CDE90588CDE90388CDE90C
:100B600001888DF80470CDE902400D980E9A002896
:100B70008DF8102003D100984946FFF765FB01F07E
:100B8000E1FF0790504601A90022002305F0F0FA8A
:100B90002846012100F028FF0028A7D140F6541074
:100BA0000121C2F2000000F01FFF002868D040F6CB
:100BB000541540F2502B0AAE08AF4FF00009C2F2B4
:100BC0000005C2F2000B00BF2846012132463B4619
:100BD00000F01EFF00284DD1DDE90C0132464FF038
:100BE0000208002818BF04320428A0F10400146889
:100BF00008BF4FF00308B0FA80F0022918BF4FEA8F
:100C00005018DBF8042020461AB15FFA88F120461C
:100C10009047DBF80C1019B92CE000BF096949B303
:100C20000A78012A04BF4A688242F7D1D1F808A0A5
:100C3000BAF1000F1ED0CDF81C90CDE90599CDE991
:100C40000399CDE901998DF80480CDE902400D9812
:100C50000E9A00288DF8102003D100983946FFF72E
:100C6000F3FA01F06FFF0790504601A9002200231C
:100C700005F07EFA2846012100F0B6FE0028A3D137
:100C800011B0BDE8F08F00002DE9F0418AB00446B4
:100C900040F25020C2F200000078012803D1012C5C
:100CA00003D9FF2094E0FD2092E001F0FE0002282D
:100CB00002D00BB9FE208BE0DDF840C0BCF1080F7C
:100CC00001D9FF2084E040F6541540F62C16002090
:100CD000012CC2F20005C2F2000618BF0546002C26
:100CE00018BF2E4696B10329CDE90800CDE90600CC
:100CF000CDE90400CDE9020069D8DFE801F002097E
:100D00000C1100200DF1080E00210EE0FE205FE026
:100D100002A8002106E0022100200DF1080E04E0E7
:100D200002A8022100F1040E0420CEF8002004AA3B
:100D3000002B82E803104FF000008DF81C0018BF54
:100D4000BCF1000F05D002A8194662461830FFF723
:100D50007BFA304600F0F6FE38B102A901AB30460E
:100D600001F1180200F06AFD78B341F2CC0104EB06
:100D7000C410C2F2000101EBC002D2F80004D2F8A4
:100D80000434013000F01F00984201D1FF201FE021
:100D900004EBC41302F5806801EBC301D8F80030FE
:100DA000DDE906C4DDE9025EDDE904725E018D5114
:100DB00001EB43114C61C1E9032CC1E901E7DDE915
:100DC0000823C1E90623C8F80000002000E0FF2046
:100DD00040B20AB0BDE8F081002904BF6FF0010005
:100DE000704780B582B00B790A6800934B1D0021D3
:100DF000FFF74AFF02B080BD2DE9F04F89B041F204
:100E0000CC0740F62C1A0DF10409E84609F1180B3D
:100E1000C2F20007C2F2000AD7F80004D7F804149F
:100E200088422BD0504600F08DFE00281EBFD7F818
:100E30000004D7F80414884220D0D7F804040DF138
:100E4000040C410107EB4010061D79586CCE446933
:100E500006948CE86E005A464346D0E90610CDE968
:100E600007104946D7F80404013000F01F00C7F806
:100E70000404504600F0E2FC0028CDD040F6541A9D
:100E80000DF10408E946C2F2000A00BFD7F80808CD
:100E9000D7F80C1888422DD0504600F053FE002899
:100EA0001EBFD7F80808D7F80C18884222D0D7F808
:100EB0000C080DF1040C07EB401000F581665ECEC6
:100EC000D0F81C5406958CE85E005A464B46D0F884
:100ED0002014D0F82404CDE907104146D7F80C08B7
:100EE000013000F01F00C7F80C08504600F0A6FCC7
:100EF0000028CBD009B0BDE8F08F000006F07CB927
:100F000005F09ABE2DE9F04105F040F84FF47A78EB
:100F1000B8FBF0F507F054FC4EF2180705FB00F69D
:100F2000CEF200073C6807F04BFC68433968864204
:100F300000FB08F008BF214657F8042C00F57A7032
:100F400001FB08F10132B1FBF2F1401A0021BDE8CA
:100F5000F081000040F63C3240F6F4210128C2F254
:100F60000002C2F2000118BF0022002818BF11467B
:100F7000084670470068016811F0100F08BF7047FD
:100F800081B0002103230091016800914168009124
:100F900044F60001C4F2000101F54C42904208BF42
:100FA0000123884240F2E85108BF0023C2F2000149
:100FB00003EBC30001EB80000099006A002801B038
:100FC00000D0004770470000FEE7000040F62C10FC
:100FD000C2F2000000F0CCBD40F62C10C2F20000BE
:100FE00000F0C6BD40F62C10C2F2000000F0C0BDFB
:100FF00040F65410C2F2000000F0BABD40F65410A2
:10100000C2F2000000F0B4BD2DE9F04381B02DED37
:10101000068B80460D469146FE20B8F1000F18BFA2
:10102000002D00F05881D8E900010024B9EB000040
:1010300064EB0101FFF7ECF99FEDAA0A01EE100A3B
:1010400081EE001A9FEDA80A11EE100A88ED021A2F
:10105000C8E9009400F0FF40B0F1FF4F0BD0B5EEAF
:10106000C01AF1EE10FA06DD9FEDA00AB4EEC01A28
:10107000F1EE10FA02DA88ED020A08E09FED9C0A10
:10108000B4EEC01AF1EE10FAC8BF88ED020A98F863
:1010900010002F78B84238D0042F10D104280ED079
:1010A0004846FFF7C9F8FFF7BDF8022121EA4000E2
:1010B000013800EE100AB8EEC00A88ED0D0A98F962
:1010C000110001281FDB9FED8B8A0026002400BF42
:1010D000C6EB061008EB8000483004F0DFFA08EB9E
:1010E0004616B0EE480A06F5C67003F00FFB06F58B
:1010F0000370B0EE480A03F009FB98F911000134BF
:10110000E6B28642E4DB88F81070052F07D0012F85
:101110000ED19FED780A0020C8E9050076E06868E6
:101120009FED740AC8F81400A868C8F818006DE0AC
:1011300098ED0C0A98EDB71A31EE408AB0EE480AE5
:1011400007F01EFEB0EE409AB0EE480A07F0E4FE4B
:1011500095ED011A95ED022A29EE013A29EE024A8F
:1011600000EE423A00EE014A88ED053A88ED064A63
:1011700098F8100006284BD89FED5E0ADFE800F0D3
:101180004646041122464400D8ED021A98ED0C0A96
:10119000D8EDB70A9FED571A08F59C7004F07EF958
:1011A00034E098ED0C0A9FED572AD8ED021AD8EDDD
:1011B000B70A9FED501A08F59C7030EE020A04F051
:1011C0006DF923E09FED480A98ED0D8A01EE109A23
:1011D000B8EE411A21EE000A07F09EFE9FED461A76
:1011E00020EE010A07F0C5FD9FED441A9FED442A49
:1011F00030EE010AB4EEC20AF1EE10FAC8BFB0EE4A
:10120000420A28EE000A01E095ED030A88ED070A7C
:1012100098F911309FED3C0A08F1120008F1140111
:1012200008F1380204F076F898F91100012851DB32
:101230009FED308A9FED35AA0024002508EB0410AD
:1012400008EB441690EDA80A06F5C67003F0DAF92B
:1012500098F8101008EB8407B0EE401A07F1380038
:101260004A1E052A12D2D8ED021A90ED000AC4EBEC
:101270000411F0EE410AB0EE481A08EB810101F1C9
:10128000480004F00BF9B0EE409A09E031B10629AC
:1012900004BF90ED000A80EE0A9A01E0B0EE489A91
:1012A00006F50370B0EE490A03F0ACF987EDA30A26
:1012B000D8F80C00D0ED1F0A07F52370B1EE600AD4
:1012C00000F038F998F911000135ECB28442B5DB31
:1012D000002000E0002040B2BDEC068B01B0BDE86C
:1012E000F08300BF00007A446F12833A6F12033A12
:1012F000CDCC4C3D00000000CDCC4C3E9A99193F1E
:10130000CDCC4C3FAB611C3F0000FA4300C0DA4536
:101310002DE9F04F81B02DED028B0446B0EE408AEE
:101320008A46BCB1FFF7FAF90020C4F80CA0FC27EC
:1013300020749AF86010062900F27B804FF00108B3
:101340000420DFE801F0040F090409760C000420F2
:10135000884607E0FE276CE00846884602E04FF02A
:10136000050801204FF0000B0AF120090025002795
:101370006074C4E900BBC4F808B000BFC5EB051039
:101380000021B0EE480A4A4604EB8000483004F0E1
:101390003BF9DAED190A04EB4516B0EE480A06F5FA
:1013A000C67003F05FF9DAED1A0A06F50370B0EEC5
:1013B000480A03F057F904EB05100137C0E9A7BB51
:1013C000C0E9A9BBFDB294F911008542D6DB04F552
:1013D0009C700AF140020021B0EE480A002704F098
:1013E00013F904F11200414604F04EF8C4E9057700
:1013F000E76194F9110001281BDB0022002100BFE6
:1014000004EB82020131C2F88C72CAB28242F7DB6D
:1014100001280DDB00250026E068284403F060FA6F
:1014200094F91100013608358642F5DB002700E00B
:10143000002778B2BDEC028B01B0BDE8F08F000050
:10144000B0B5044634B394F91110012922DB002011
:10145000002500BF04EB8002106A20B192EDA30AC0
:1014600003F0ACFA617C01354AB2E8B29042F1DB9C
:10147000012AB8BFB0BD0020002500BF04EB8000EA
:10148000006A10B103F07EF9617C01354AB2E8B21E
:101490009042F3DBB0BD000070B5044694F9110032
:1014A000012822DB00260025E06800EBC60003F0DF
:1014B000F1FAE06800EBC60003F0ECF904EB8601FA
:1014C0000028086214D004EB061100F1080601356B
:1014D0004CCE406901F5277C8CE84C00C1F8A8028D
:1014E000EEB294F911008642DEDB002040B270BDFE
:1014F000FE2040B270BD0000B5EEC01A30EE600AAA
:10150000F1EE10FAD8BF7047B6EE002A21EE022A9B
:10151000B4EEC20AF1EE10FAC4BF30EE410A7047D1
:10152000B1EE422AB4EEC20AF1EE10FAB8BF30EEC4
:10153000010A704790ED001AB4EEE01AF1EE10FACD
:10154000C4BFC0ED000AB0EE601AB4EEC01AF1EEEE
:1015500010FAB8BF80ED000A7047000040F2180092
:10156000C2F200007047000040F20040C2F20000EA
:1015700000F052BF40F29040C2F2000000F04CBFB9
:1015800040F2A000C2F2000000F046BF40F2A030DE
:10159000C2F2000000F040BF40F20010C2F20000B2
:1015A00000F03ABF40F24050C2F2000000F034BFF9
:1015B00010B5002802BFFE2460B210BD0024342103
:1015C00000F8244BFEF759FE60B210BDB0B50446DA
:1015D000002C02BFFE2040B2B0BD254655F8100FCA
:1015E00001466FF3DF21A1F5B671B1F5A56F11D8F2
:1015F000C0F3CA21A1F5B671B1F5A56F0AD8A988C3
:10160000800D40EA81206FF3DF20A0F5B670B0F5C1
:10161000A56F02D9FF2040B2B0BDC1F34A02FF203E
:1016200011F4405F00F0C28089B2B1F5804FC0F084
:10163000BD80A2F5B671B1F5A56F00F2B7800120AB
:101640002070FFF75FFCC4E9020104F1340024219B
:10165000FEF713FE2968A8889FED550A8A0DC1F38D
:10166000CA236FF3DF2101EE101A42EA802202EE54
:10167000103AB8EE411AC0F34A016FF3DF22B8EE18
:10168000422A31EE003A9FED4B1A04EE102A05EE85
:10169000101A32EE002A810BB8EE444A33EE033AB8
:1016A000B8EE455A32EE022A34EE004A35EE005AC0
:1016B00083EE013A82EE012A84ED0B3A34EE043ACD
:1016C00035EE054A84ED0C2A83EE012A84EE013AB8
:1016D00084ED092A84ED0A3A84F83910C0F3013008
:1016E00084F83800E08A6087208BA087608BE087D1
:1016F000207F002818BF012084F84000617F002966
:1017000018BF012184F84110E28B02F0010384F834
:101710004230C2F3400384F84330C2F3800384F8BC
:101720004430C2F3C00384F84530C2F3001384F898
:101730004630C2F3401384F84730C2F3801384F874
:101740004830C2F3C01384F84930C2F3002384F850
:101750004A30C2F3402384F84B30C2F3802384F82C
:101760004C30C2F3C02384F84D30C2F3003384F808
:101770004E30C2F3403384F84F30C2F38033D20B83
:1017800084F8503084F8512084F8520084F85310C3
:10179000208C02EE100A0020B8EE422A32EE000A37
:1017A00030EE000A80EE010A84ED0D0A40B2B0BDB1
:1017B000000080C40000A54410B504460020FFF7D7
:1017C000C9FB04F11001122202F056FE002818BFD6
:1017D0004FF0FF3010BD000080B50246012001210E
:1017E00004F09EFD0138B0FA80F0400980BD000091
:1017F00070470000012001F0B3B80000102001F094
:10180000AFB80000202001F0ABB8000072B600BFF6
:10181000FEE7000090F82020013AD2B2012A04D855
:10182000006800F11402002004E000F1240201200D
:101830004FF48021136819431160704710B590F878
:101840002040D0F800C0DCF808E0013CE4B2012CF4
:101850000ED81EF0E05F11D0CEF301600124844069
:101860001C60D1E9023E7BB14C6843EAC4030DE041
:1018700000F1240301204FF4802123E000F1240330
:1018800001204FF400111DE00B685B050CEB00100C
:1018900043EA0E03C0F880310B69C0F8843100F5CB
:1018A000C073097D012901BF00F5C2710C6844F4C1
:1018B00080740C605168C0F88C111168C0F88811F0
:1018C000002001211A681143196010BD90F82020F2
:1018D000013AD2B2012A2ED8B0B546F20060C4F265
:1018E0000000026842F001020260026822F47C52A9
:1018F00002604A6A036843EA0222012302604C69DB
:1019000004F01F0203FA02F2C3696FEA020C934368
:10191000C361CB69012B14D043BBC36800EBC40E79
:1019200003EA0C03C360CB688D8845EA0343CEF815
:1019300040308E4612E0416A41F48021416201202C
:101940007047C36800EBC40E1343C3600D688B88F7
:1019500043EA0543CEF8403001F10C0E00EBC4031E
:101960008C68BEF8005045EA04455D648B694568A3
:1019700045EA0204002B08BF05EA0C0444600B6929
:10198000456945EA0204002B08BF05EA0C044461DE
:10199000096A0129BDE8B04002BFC1691143C161B4
:1019A000016821F00101016000207047D0B100689A
:1019B00046F20041C4F20001884208D046F6000118
:1019C000C4F20001884218BF7047012000E00020E7
:1019D00040F250213422C2F2000110FB0210006CD0
:1019E00000B100477047000090F82020013AD2B2C1
:1019F000012A84BF002070470068002900F110020E
:101A000008BF00F10C02106800F0030070470000EE
:101A100010B590F82040013CE4B2012C0DD8D0F86C
:101A200000C081B1DCF8104014F0030F10D100F1B8
:101A3000240201204FF400117AE000F12402012079
:101A40004FF4802174E0DCF80C4014F0030F73D0E5
:101A50000CEB011CDCF8B0410CF5D87E14F004044A
:101A60009460DCF8B04102D1640D146001E0E40838
:101A70005460DEF800400CF5DA7E04F00204D46015
:101A8000DCF8B44114F0080F06BFDEF8004004F0A3
:101A90000F04082400291461DEF80040C4F3072471
:101AA0009461DEF800404FEA14445461DCF8B82138
:101AB0001A70026802EB0112D2F8B8214FEA122222
:101AC0005A70026802EB0112D2F8B8214FEA1242B2
:101AD0009A70026802EB0112D2F8B8214FEA126242
:101AE000DA70026802EB0112D2F8BC211A710268A6
:101AF00002EB0112D2F8BC214FEA12225A7102689D
:101B000002EB0112D2F8BC214FEA12429A7102682C
:101B100002EB01124FF02001D2F8BC214FEA126211
:101B2000DA71006800F1100208BF00F10C02002019
:101B300013681943116010BD00F1240201204FF415
:101B40000011F5E790F820100139C9B2012984BFCE
:101B50000020704700688168C1F380618268C2F329
:101B6000C06280681144C0F30070084470470000F0
:101B70002DE9F04F81B0044620684669D0F8049002
:101B80008768D0F80CB0D0F810A0D0F8188016F004
:101B9000010F03D1002530071CD423E0F90710D032
:101BA00001218160B80709D4780700F198803807CF
:101BB00000F19B80204600F009FB02E0204600F087
:101BC00023FB0025F80500F19580F80300F1B580AE
:101BD000300707D51BF010001FBF20681021C1601F
:101BE00045F40075700708D51BF0080005D0206883
:101BF0000821C160204600F025FAB00707D520680B
:101C0000C06810F0030F1CBF204600F039FA7006C0
:101C100007D51AF010001FBF20681021016145F49C
:101C20008065B00608D51AF0080005D020680821A4
:101C30000161204600F042FAF00607D520680069ED
:101C400010F0030F1CBF204600F056FAB00308D571
:101C500019F0100005D0206810214160204600F0E6
:101C600069FAF00308D519F0080005D020680821AA
:101C70004160204600F05EFB300440F198805FEA4E
:101C8000497040F1918006F4807018F0020F08EA64
:101C9000102040EA0500014618BF41F0020116F489
:101CA000007F08BF014618F0040F0D4618BF45F02D
:101CB000040516F4806F08BF0D4616F4006F18BFB8
:101CC00018F0700070D010380009052867D8DFE8D8
:101CD00000F003585B5E616445F008055FE04FF477
:101CE0000065F8057FF571AF04E04FF48055F80505
:101CF0007FF56BAF20684FF480718160B8050AD41E
:101D000078050FD4380513D4204600F09BFAF80369
:101D10007FF55EAF11E0204600F0B2FAF8037FF5E0
:101D200057AF0AE045F40055F8037FF551AF04E0E2
:101D300045F48045F8037FF54BAF20684FF48031C0
:101D40008160B8030AD478030FD4380313D4204633
:101D500000F0B4FA30073FF53DAF43E7204600F00E
:101D6000CBFA30073FF536AF3CE745F40045300786
:101D70003FF530AF36E745F4803530073FF52AAF01
:101D800030E745F010050AE045F0200507E045F092
:101D9000400504E045F0800501E045F480752068C9
:101DA000816921F070018161206804214160002D6A
:101DB00004BF01B0BDE8F08F606A2843606220462E
:101DC00001B0BDE8F04FFFF7F1BD0000B0B504462B
:101DD000002C04BF0120B0BD94F8200010B92046AB
:101DE00000F076F82068016841F00101016000F020
:101DF000A9FE05462068416811F0010F05D100F0E9
:101E0000A1FE401B0B28F5D310E0016821F0020170
:101E1000016000F097FE05462068416811F0020F4E
:101E20000DD000F08FFE401B0B28F5D3606A052112
:101E300040F400306062012084F82010B0BD217EA3
:101E4000026822F08003012908BF42F0800303608A
:101E5000617E026822F04003012908BF42F040037E
:101E60000360A17E026822F02003012908BF42F02E
:101E700020030360E17E026842F01003012908BFDD
:101E800022F010030360217F026822F00803012979
:101E900008BF42F008030360617F026822F0040378
:101EA000012908BF42F004030360D4E901C2D4E968
:101EB000033561691A432A431143ACF1010211430E
:101EC000C16100200121606284F82010B0BD0000D3
:101ED00080B586B0002246F6000143F6400C05921C
:101EE000CDE90322CDE90122C4F20001C4F2020CC3
:101EF000036840F20040C4F202008B4252D046F226
:101F00000041C4F200018B4240F09A8040F2E0515F
:101F1000C2F200010A68531C002A0B600DD1002197
:101F20000091DCF8001041F00071CCF80010DCF8F2
:101F3000001001F00071009100990021022300F5CA
:101F4000006000915CF8102C42F008024CF8102C54
:101F50005CF8102C02F008020092009A0322019211
:101F6000CDE9023109210492059101A900F004FD97
:101F700013200521002200F065FE132000F052FE20
:101F800014200521002200F05DFE142000F04AFE1E
:101F900015200521002200F055FE152000F042FE1C
:101FA00006B080BD0092DCF8001041F08061CCF8F2
:101FB0000010DCF8001001F080610091009940F2FF
:101FC000E051C2F200010A68531C002A0B600DD1D7
:101FD00000210091DCF8001041F00071CCF80010F5
:101FE000DCF8001001F000710091009900210091CF
:101FF0005CF8102C42F002024CF8102C5CF8102C0B
:1020000002F002020092009A602201920222CDE9BF
:102010000221032104910921059101A900F0ACFCE2
:1020200040200521002200F00DFE402000F0FAFDC6
:1020300041200521002200F005FE412000F0F2FDC4
:1020400006B080BDD0B1006846F20041C4F2000184
:10205000884208D046F60001C4F20001884218BF49
:102060007047012000E0002040F250213422C2F2EB
:10207000000110FB0210C06A00B100477047000069
:10208000D0B1006846F20041C4F20001884208D095
:1020900046F60001C4F20001884218BF70470120D3
:1020A00000E0002040F250213422C2F2000110FB77
:1020B0000210806A00B1004770470000D0B100688C
:1020C00046F20041C4F20001884208D046F6000101
:1020D000C4F20001884218BF7047012000E00020D0
:1020E00040F250213422C2F2000110FB0210406B7A
:1020F00000B1004770470000D0B1006846F20041CF
:10210000C4F20001884208D046F60001C4F2000182
:10211000884218BF7047012000E0002040F25021A3
:102120003422C2F2000110FB0210006B00B1004724
:1021300070470000D0B1006846F20041C4F20001CF
:10214000884208D046F60001C4F20001884218BF58
:102150007047012000E0002040F250213422C2F2FA
:10216000000110FB0210806B00B1004770470000B7
:10217000B0B5044694F8200001281ED1022084F84E
:1021800020002068016821F00101016000F0DAFC04
:10219000054600BF2068406810F0010F13D000F022
:1021A000D1FC401B0B28F5D3606A40F4003060621C
:1021B000052084F820000120B0BD606A40F40020B2
:1021C00060620120B0BD00206062B0BDD0B1006887
:1021D00046F20041C4F20001884208D046F60001F0
:1021E000C4F20001884218BF7047012000E00020BF
:1021F00040F250213422C2F2000110FB0210C069EB
:1022000000B1004770470000D0B1006846F20041BD
:10221000C4F20001884208D046F60001C4F2000171
:10222000884218BF7047012000E0002040F2502192
:102230003422C2F2000110FB0210006900B1004715
:1022400070470000D0B1006846F20041C4F20001BE
:10225000884208D046F60001C4F20001884218BF47
:102260007047012000E0002040F250213422C2F2E9
:10227000000110FB0210006A00B100477047000027
:10228000D0B1006846F20041C4F20001884208D093
:1022900046F60001C4F20001884218BF70470120D1
:1022A00000E0002040F250213422C2F2000110FB75
:1022B0000210406900B1004770470000D0B10068CB
:1022C00046F20041C4F20001884208D046F60001FF
:1022D000C4F20001884218BF7047012000E00020CE
:1022E00040F250213422C2F2000110FB0210406A79
:1022F00000B1004770470000D0B1006846F20041CD
:10230000C4F20001884208D046F60001C4F2000180
:10231000884218BF7047012000E0002040F25021A1
:102320003422C2F2000110FB0210806900B10047A4
:1023300070470000D0B1006846F20041C4F20001CD
:10234000884208D046F60001C4F20001884218BF56
:102350007047012000E0002040F250213422C2F2F8
:10236000000110FB0210C06B00B100477047000075
:1023700070B50446A66D00F0E5FB054694F83500FF
:10238000022825D12068016821F016010160416909
:1023900021F080014161216C09B9A16C19B101687A
:1023A00021F008010160016821F00101016000E0F5
:1023B0002068006810F0010F0ED000F0C3FB401B36
:1023C0000528F5D920206065032084F835000CE04D
:1023D00080206065012008E0E06D3F2101FA00F0F7
:1023E000B060012084F8350000200021C0B284F8DC
:1023F000341070BD90F8351002291FBF802141654F
:1024000001207047052180F835100068016821F02F
:102410000101016000207047F0B581B00446002042
:1024200048F2B5130821009040F21400C1F64E3373
:10243000C2F200000268D4E9166037688140A2FB4E
:10244000032539420DD02268136813F0040F08D019
:10245000136823F004031360B160616D41F0010162
:10246000616501218140394209D02268526912F028
:10247000800F1FBFB160616D41F0020161650421F1
:102480008140394209D02268126812F0020F1FBF42
:10249000B160616D41F004016165102181403942F4
:1024A0001AD02068026812F0080F15D0B1600268D7
:1024B000016812F4802F06D1C9055EBF016821F0C2
:1024C0000801016001E0080301D4216C00E0A16C67
:1024D00000291CBF20468847E16D202000FA01F248
:1024E0003A4242D02068036813F0100F3DD0B2602A
:1024F00094F835300268052B1ED122F016020260D6
:10250000426922F080024261226C0AB9A26C1AB1BF
:10251000026822F0080202603F208840B06001207B
:1025200084F83500002084F83400216D00293FD064
:102530002046884701B0F0BD016852030CD4C9059C
:102540000ED4016821F010010160012084F83500EB
:10255000002084F8340003E0080301D4616C00E03B
:10256000E16B00291CBF20468847606D00B3606D99
:1025700010F0010F17D00521A80A84F83510216842
:102580000A6822F001020A60009A01328242009237
:1025900003D80A6812F0010FF6D1012084F8350043
:1025A000002084F83400E16C00291CBF20468847D5
:1025B00001B0F0BD2DE9F041044600F0C3FA054634
:1025C000002C02BF0126F0B2BDE8F081022084F8A1
:1025D0003500002084F834002068016821F00101F2
:1025E000016000E02068016811F0010F08D000F0E0
:1025F000A9FA401B0528F5D903252023032667E007
:10260000016848F23F02CFF2100201EA020CD4E95D
:102610000126D4E90353D4E90578D4E9071E42EA38
:102620000C0232432A431A433A4342EA0802114356
:10263000626A41EA0E01042A1DD1D4E90B3719431D
:1026400039430160014651F8143F23F00703134357
:10265000D4E90A2E42EA030CBEF1000F13D0B8F5FC
:10266000005F3BD0B8F1000F4BD1022A4CD0012AB9
:1026700040D042B948E00160014651F8143F23F0D0
:10268000070343EA020C4AF6AB22C1F800C06FF020
:102690000F010125002651FA80F1CAF6AA22A1FBFA
:1026A00002235F294FF03F014FEA131249F27C43A6
:1026B000C0F600039A5C40F2FF3320EA03004FF0BB
:1026C000000388BF40F004009140C4E91602816015
:1026D000F0B2636584F83550BDE8F081032AD2D8A2
:1026E0000125402306EB82070126DFE802F0020DF8
:1026F0000203EDE7AEF1C072B2FA82F252093AB9C2
:10270000C1E7032A04D3BED1CEF30062002ABAD0B7
:10271000012540230126DBE710B590F834C0BCF159
:10272000010F48D04FF0010CD0F858E080F834C0C9
:1027300090F835C0BCF1010F3AD14FF0020C80F88F
:1027400035C04FF0000CC0F854C0D0F800C0DCF821
:10275000004024F48024CCF80040CCF80430836896
:10276000402B0B4608BF1346CCF8083008BF0A467A
:10277000CCF80C203F22C16D02FA01F1CEF808100E
:10278000DCF8001041F01601CCF80010006C0028B5
:102790001EBFDCF8000040F00800CCF80000DCF8B8
:1027A000000040F00100CCF800000020C0B210BDD5
:1027B000002180F834100220C0B210BD10B50446CC
:1027C00014F0010F36D1A0073ED4600746D420078D
:1027D0004ED4E00656D4A0065ED4600666D4200629
:1027E0006ED4E00577D4A00500F18080600500F18B
:1027F0008880200500F19080E00400F19880A0041A
:1028000000F1A080600407D540F2A050C2F20000A1
:10281000806B002818BF8047200458BF10BD40F2CD
:10282000A050C2F20000C06B002800F09780BDE805
:102830001040004740F2A050C2F20000006800289B
:1028400018BF8047A007C0D540F2A050C2F20000D8
:102850004068002818BF80476007B8D540F2A050F4
:10286000C2F200008068002818BF80472007B0D55A
:1028700040F2A050C2F20000C068002818BF804794
:10288000E006A8D540F2A050C2F20000006900287E
:1028900018BF8047A006A0D540F2A050C2F20000A9
:1028A0004069002818BF8047600698D540F2A050C4
:1028B000C2F200008069002818BF8047200690D52A
:1028C00040F2A050C2F20000C069002818BF804743
:1028D000E0057FF588AF40F2A050C2F20000006A28
:1028E000002818BF8047A0057FF580AF40F2A050B8
:1028F000C2F20000406A002818BF804760057FF5DB
:1029000078AF40F2A050C2F20000806A002818BFE1
:10291000804720057FF570AF40F2A050C2F2000062
:10292000C06A002818BF8047E0047FF568AF40F216
:10293000A050C2F20000006B002818BF8047A0041E
:102940007FF560AF40F2A050C2F20000406B00285B
:1029500018BF804760043FF557AF5DE710BD00002A
:1029600043F61441C4F201010A6802421CBF086028
:10297000FFF724BF704700002DE9F04F82B041F609
:102980000042082743F6004B4FF0010E00250024BB
:102990004FF00008C4F20202C4F2010B904200F1B1
:1029A0003E4202F1FF7208BF07274FEAB223072B0E
:1029B00038BF4FEAB22700970AE000BF08F10108CC
:1029C00004350234B8F1100F04BF02B0BDE8F08F37
:1029D0000E680EFA08FC16EA0C0FEFD0D1F804903E
:1029E00009F0030AAAF10106012E17D8D0F808E071
:1029F000CB68032202FA04F62EEA0606A3404FF043
:102A0000010E33438360C9F30013466803FA08F3E9
:102A100026EA0C063343436003E000BFBAF1030F1C
:102A200023D0C6680322BAF1020F02FA04F326EAA1
:102A300003038E6806FA04F643EA0603C36014D162
:102A400005F01C030F2202FA03F64FF6FC72C7F6DC
:102A5000FF7202EA58020244176AB7430E6906FA87
:102A600003F33B431362D1F804900768032309F092
:102A7000030219F4403F03FA04F302FA04F227EACE
:102A8000030342EA0302026098D0002205F00C071B
:102A90000F26019243F64402BE40C4F202021346DE
:102AA0001A6842F480421A601A6802F48042019265
:102AB00028F00302019B5A444FF60843CFF6FF73F8
:102AC000994652F80930B343009E06FA07F73B4394
:102AD00042F80930DBF808204B6822EA0C0213F4B4
:102AE000801F18BF42EA0C0213F4001FCBF8082025
:102AF00043F60C42C4F201021646326822EA0C0286
:102B000018BF42EA0C0213F4003F3260DBF80420E5
:102B100022EA0C0218BF42EA0C0213F4803FCBF801
:102B20000420DBF8002022EA0C0218BF42EA0C0263
:102B3000CBF8002042E70000002A08BF09048161A9
:102B40007047000040F20800C2F200008068704741
:102B500040F20800C2F200000178826811448160EE
:102B60007047000080B543F60040C4F202000168DF
:102B700041F400710160016841F480610160016805
:102B800041F480710160032000F08EF80F2000F006
:102B900005F800F025F8002080BD000070B540F277
:102BA000080604464FF47A71C2F200063078B1FB91
:102BB000F0F040F21401C2F200010968B1FBF0F03C
:102BC00000F07AFC01250F2C08D838B94FF0FF30FF
:102BD00021460022002500F035F87460284670BDBB
:102BE00082B043F6400100200190C4F202014A681D
:102BF00042F480424A604A6802F480420192019A9B
:102C000000900868002240F08050086008680F219A
:102C100000F08050009000986FF0010002B000F0CA
:102C200011B800000028B8BF704700F01F01012252
:102C3000400902FA01F14EF20012CEF2000242F80F
:102C40002010704710B500F00F034EF60C5E00F137
:102C5000604CB0F1FF3FA3F10403CEF2000E7344C9
:102C600003F10C04C8BF0CF56444DEF80000C0F3A7
:102C7000022000F1040CC31E80F00700BCF1070F16
:102C80004FF0010C38BF0023042828BF04200CFAA1
:102C900000F0013808400CFA03F10F319840114060
:102CA00008430001207010BD4EF60C514FF6FF0393
:102CB000CEF200010A681A4060F30A2242F08060F6
:102CC00040F0FD70086070472DE9F04104460D4664
:102CD000002C00F0A78043F60808C4F20208D8F8D8
:102CE000F80300F00700A84208D288F8F853D8F893
:102CF000F80300F00700A84240F09480206810F02C
:102D0000020F17D0410742BFD8F8001041F4E0513C
:102D1000C8F80010010742BFD8F8001041F4604124
:102D2000C8F80010D8F80010A26821F0F001114393
:102D3000C8F80010C00734D06068811E022905D28F
:102D400058F8081C11F0007F6CD00CE0012805D168
:102D500058F8081C11F4003F64D004E058F8081C2F
:102D600011F0020F5ED0D8F8001021F003010843E3
:102D7000C8F80000FFF7E6FE064641F2883700BFBC
:102D8000D8F80000616800F00C00B0EB810F08D0AB
:102D9000FFF7D8FE801BB842F2D90320C0B2BDE8CD
:102DA000F081D8F8F80300F00700A84207D988F8A6
:102DB000F853D8F8F80300F00700A84232D1206891
:102DC00010F0040F07D0D8F80010E26821F4E051A9
:102DD0001143C8F80010000708D5D8F80000216991
:102DE00020F4604040EAC100C8F8000000F046F856
:102DF000D8F8001049F2F832C0F60002C1F303110E
:102E0000515CC84040F21401C2F20001086040F277
:102E10000C00C2F200000068FFF7C0FE0020C0B244
:102E2000BDE8F0810120C0B2BDE8F08140F214009D
:102E300043F6080149F20842C2F20000C4F202015E
:102E4000C0F6000200680968C1F38221515CC840E5
:102E50007047000040F2140043F6080149F20842AE
:102E6000C2F20000C4F20201C0F600020068096864
:102E7000C1F34231515CC8407047000010B543F6C1
:102E80000404C4F20204606800F00C0008280BD0AF
:102E900004281EBF42F20040C0F2F40010BD41F60B
:102EA0000030C0F2B70010BD2268206841F6003142
:102EB0000023C0F2B70110F4800F02F03F0204BFFC
:102EC00042F20041C0F2F4012068C0F38810A1FB77
:102ED0000001FDF775F921680222C1F3014102EBFF
:102EE0004101B0FBF1F010BD2DE9F04782B004467E
:102EF000002C3FD0207843F6000A43F67007C4F256
:102F0000020AC4F20207C0073FD057F8680C00F06D
:102F10000C00042830D057F8680C00F00C0008288A
:102F200004D157F86C0C10F4800F25D16668B6F503
:102F3000803F09D0DAF80000B6F5A02F40F072818A
:102F400040F48020CAF80000DAF8000040F4803035
:102F5000CAF80000FFF7F6FD054600BFDAF80000EA
:102F600010F4003F11D1FFF7EDFD401B6428F5D9A7
:102F7000032098E1012096E1DAF8000010F4003F08
:102F800003D06068002800F0D480207840F2000868
:102F9000C4F24728800737D557F8680C10F00C0F9B
:102FA00020D057F8680C00F00C00082804BF57F830
:102FB0006C0C10F4800F15D0E068002800F0A5809C
:102FC0000120C8F80000FFF7BDFD0546DAF8000053
:102FD00010F0020F0FD1FFF7B5FD401B0228F5D905
:102FE000032060E1DAF8000010F0020F1CBFE06877
:102FF000012840F08880DAF80000216920F0F8000C
:1030000040EAC100CAF800002078000725D56069B1
:1030100088B10120C8F8800EFFF794FD054600BF77
:10302000786810F0020F18D1FFF78CFD401B0228C2
:10303000F6D9032037E10020C8F8800EFFF782FDA3
:10304000054600BF786810F0020F06D0FFF77AFD42
:10305000401B0228F6D9032025E12078400740F1E3
:103060008C8057F8300C4FF0000910F0805F0FD1C2
:10307000CDF804904FF0010957F8300C40F0805023
:1030800047F8300C57F8300C00F080500190019850
:1030900043F60006CFF6FE765AF8060010F4807F5D
:1030A00014D15AF8060040F480704AF80600FFF781
:1030B00049FD05465AF8060010F4807F06D1FFF757
:1030C00041FD401B0228F5D90320ECE0A668012E43
:1030D00005D03868052E2ED140F0040038603868DD
:1030E00040F001003860FFF72DFD054641F28836BB
:1030F000386810F0020F37D1FFF724FD401BB042B3
:10310000F6D90320CFE00120CDE00020C8F8000070
:10311000FFF718FD054600BFDAF8000010F0020FB7
:103120003FF472AFFFF70EFD411B03200229F3D9D4
:10313000B9E00120B7E020F001003860386820F0E5
:1031400004003860FFF7FEFC0546002ECED141F2A8
:103150008836386810F0020F06D0FFF7F3FC411BE9
:103160000320B142F5D99EE0B9F1010F02BF57F833
:10317000300C20F0805047F8300CA669002E00F08B
:10318000918057F8680C00F00C00082803D1012E3C
:1031900022D1012087E00020C8F86000FFF7D2FCB0
:1031A0000546022E0CD100BFDAF8000010F0007FB7
:1031B00055D0FFF7C7FC411B03200229F4D972E068
:1031C000DAF8000010F0007F6CD0FFF7BBFC411B69
:1031D00003200229F4D966E057F86C0CE16900F489
:1031E00080028A4263D1216A00F03F028A4260D1A4
:1031F000626A47F6C0710140B1EB821F5BD1A16AE0
:103200004FF6FF72C903914300F44032A1F58031BB
:103210008A4252D1E16A00F07060B0EB016F41D098
:10322000012040E020F48030CAF80000DAF8000005
:1032300020F48020CAF80000FFF784FC0546002E29
:103240007FF48CAEDAF8000010F4003F3FF49DAE3E
:10325000FFF778FC411B03206429F3D923E004F134
:103260001C064FCE0843D90340EA82104FF6FF7286
:10327000914340EA0660A1F58031084347F86C0CA1
:103280000120C8F86000FFF75DFC0446DAF8000092
:1032900010F0007F06D1FFF755FC011B0320022927
:1032A000F4D900E00020C0B202B0BDE8F0870120F0
:1032B000F9E70120F7E70120F5E70120F3E7000037
:1032C00070B50446002C02BF0125284670BDD4F815
:1032D00024C0BCF1000F04D00021216104F11401CD
:1032E00005E06168B1F5827F03D004F11C01002282
:1032F0000A6000254FF0000EA56294F8511041B904
:10330000204684F8505000F03FF8D4E909C101F498
:10331000005E022284F851202268136823F04003E3
:103320001360D4E90130D4E9031603F4827300F486
:10333000044001F400611843084306F00201084309
:10334000616901F001010843A16901F400731843A8
:10335000E36903F038031843236A03F0800318433A
:1033600040EA0E001060042000EA11400CF0100149
:1033700008435060D06920F40060D0610120656589
:1033800084F85100284670BD2DE9F04786B000262C
:10339000044643F200070596CDE90366CDE90166D0
:1033A000C4F201072068B84202D006B0BDE8F08739
:1033B00043F63000009601AD4FF002084FF00309CC
:1033C0004FF0050AC4F20200416941F480514161A5
:1033D000416901F48051009100990096016841F023
:1033E00002010160016801F002010091009900965C
:1033F000016841F0010101602946006800F0010008
:10340000009000981820019007F55440CDE90286FD
:10341000CDF81090CDF814A0FFF7AEFA8020294621
:10342000CDE9010803A880E8400607F55040FFF702
:10343000A3FA40F2A00546F240474FF0C0694FF4AE
:1034400080684FF44030C2F20005C4F20207C5E9BB
:103450000079C5E90266C5E90486C5E90666C5E9DD
:1034600008062846FFF7A6F8002818BFFEF7CEF991
:10347000E564AC6340F2A03507F11800402100225A
:10348000C2F20005C5E9000905F1080080E806015F
:103490004FF40030C5E90522EA61C5E90802284673
:1034A000FFF788F8002818BFFEF7B0F9A564AC63F1
:1034B00006B0BDE8F0870000411E0020B0EB116FA0
:1034C0001CBF012070474EF21002F023CEF2000222
:1034D00051604EF62351CEF200010B70072190602F
:1034E00011607047704700007047000090F83C3052
:1034F0000222012B55D010B5012380F83C3080F812
:103500003D200268D2F804E0D2F808C00C682EF022
:1035100070032343536041F2FF73C4F200039A42E5
:10352000BDE810400BDC40F2FF73C4F200039A4286
:1035300013DCB2F1804F29D040F2004315E040F295
:10354000FF33C4F201039A4214DC41F60003C4F2D3
:1035500000039A421AD0002314E040F60003C4F29C
:1035600000039A4212D040F60043C4F200039A428C
:103570000CD010E044F20003C4F201039A4205D0DB
:1035800040F20043C4F201039A4204D149682CF08E
:103590008003194391600121002280F83D1080F8DA
:1035A0003C20D0B27047000010B50446002C04BF88
:1035B000012010BD94F83D0028B9002084F83C009B
:1035C000204600F0B1F8022040F6FF3284F83D00BA
:1035D000C4F200022068016890420FDCB0F1804F15
:1035E0001EBF40F20043C4F20003984217D040F6D9
:1035F0000003C4F20003984211D014E040F60043E7
:10360000C4F2000398421EBF40F20043C4F201031B
:10361000984204D00023C4F20103984203D1A36866
:1036200021F07001194341F6FF73C4F20003984280
:103630000DDC90421FDCB0F1804F1EBF40F2004213
:10364000C4F2000290423BD040F6000221E043F673
:10365000FF72C4F20102904220DC42F20002C4F286
:10366000000290421EBF0022C4F20102904227D005
:1036700040F2004220E040F60042C4F200029042D4
:103680001EBF41F60002C4F20002904218D041F67B
:103690000042C4F20002904212D015E044F200024F
:1036A000C4F2010290421EBF44F60002C4F20102BD
:1036B000904205D044F20042C4F20102904203D18C
:1036C000226921F440711143E268A36921F080016D
:1036D000C262194340F200436268C4F2010382628D
:1036E00040F480629A4204BF62690263026842F059
:1036F00004020260012242610160002084F8462039
:1037000084F83E2084F83F2084F8402084F841204B
:1037100084F8422084F8432084F8442084F845202B
:1037200084F83D2010BD000080B584B0016844F2EB
:10373000004243F64000C4F20102C4F2020091428A
:1037400018D041F20042C4F2000291421FD040F66C
:103750000002C4F20002914217D1002103910168D6
:1037600041F004010160006800F004000390039838
:1037700004B080BD00210191416841F400314160F5
:10378000406800F400300190019804B080BD002131
:1037900000220291016841F02001016005210068CA
:1037A00000F02000029002983720FFF74BFA3720F4
:1037B00004B0BDE88040FFF735BA000090F83C3017
:1037C0000222012B00F0C58080B5012380F83C3037
:1037D00080F83D204FF67772D0F800C0DCF8083052
:1037E00023EA0202CCF808200B684F2B28DC1F2BA1
:1037F00043DD202B18BF302B43D0402B40F0AB8053
:10380000D1F804E0C968DCF82030DCF8202022F090
:103810000102CCF82020DCF8182022F0F00242EA65
:103820000111CCF8181023F00A0141EA0E01CCF87E
:103830002010DCF8081021F0770141F047017DE00D
:103840006F2B26DDB3F5005F47D0B3F5805F77D0EF
:10385000702B40F08080D1E90123C9681A4342EA05
:103860000121DCF8082022F47F421143CCF8081033
:10387000DCF8081041F0770160E0002B18BF102B36
:1038800069D1DCF8081021F07701194341F00701F4
:1038900054E0502B33D0602B5DD1D1F804E0C968DF
:1038A000DCF82030DCF8202022F01002CCF82020B8
:1038B000DCF8182022F4704242EA0131CCF81810EA
:1038C00023F0A00141EA0E11CCF82010DCF808101A
:1038D00021F0770141F0670130E0D1E90123C968A7
:1038E0001A4342EA0121DCF8082022F47F42114306
:1038F000CCF80810DCF8081041F480411EE0D1F843
:1039000004E0C968DCF82030DCF8202022F0010255
:10391000CCF82020DCF8182022F0F00242EA011155
:10392000CCF8181023F00A0141EA0E01CCF820105F
:10393000DCF8081021F0770141F05701CCF80810AD
:103940000022012180F83D10002180F83C10BDE8E4
:103950008040D0B270470122F3E7000070470000BA
:10396000B0B504462068C168026901EA0205A907EA
:1039700014D56FF00201016101212177806910F0F7
:10398000030F03D02046FFF7E9FF05E0204600F0D3
:1039900075F8204600F04CFA00202077680715D50E
:1039A00020686FF00401016102212177806910F421
:1039B000407F03D02046FFF7D1FF05E0204600F00E
:1039C0005DF8204600F034FA00202077280715D54E
:1039D00020686FF00801016104212177C06910F0AF
:1039E000030F03D02046FFF7B9FF05E0204600F0A3
:1039F00045F8204600F01CFA00202077E80615D58F
:103A000020686FF01001016108212177C06910F46E
:103A1000407F03D02046FFF7A1FF05E0204600F0DD
:103A20002DF8204600F004FA00202077E80706D0A1
:103A300020686FF001010161204600F0FBF92806C3
:103A400006D520686FF0800101612046FFF74AFD2E
:103A5000680606D520686FF040010161204600F03D
:103A6000EBF9A80658BFB0BD20686FF020010161D6
:103A70002046BDE8B040FFF737BD000070470000AA
:103A800090F83C30012B02BF0223D8B270474FEAB6
:103A9000B2020123032A80F83C3000F201812DE9B3
:103AA000F041DFE802F002813EC303681E6A1A6A31
:103AB00022F0010226F002061A621A46D3F804C068
:103AC00052F8185F8F680C68374325F0730643F48B
:103AD000806546EA040E40F20046C4F20106B54293
:103AE00001BF27F00C04CF6827F004072743B54235
:103AF00001BFD1E905452CF44076264346EA050C82
:103B0000C3F804C0C3F818E04E685E631F629F6983
:103B100047F008079F619F6927F004079F610969C3
:103B2000B8E003681F6A1A6A22F4807227F40077EB
:103B30001A621A46D3F804C052F81C4F8E680D68FA
:103B400047EA062E40F2004624F0730444EA0508D2
:103B500043F48065C4F20106B54209D1CF6840F252
:103B6000FF443F0227EA04042EF4406744EA070EAC
:103B7000B54201BFD1E905452CF4405747EA041787
:103B800047EA051CC3F804C0C3F81C804F68DF6314
:103B9000C3F820E0DF6947F00807DF61DF6927F03D
:103BA0000407DF61096975E003681F6A1A6A22F079
:103BB000100227F020071A621A46D3F804C052F800
:103BC000184F8E680D6847EA061E40F2004624F43E
:103BD000E64444EA052843F48065C4F20106B54290
:103BE00001BFCF686FF04F0404EA07142EF0C0073E
:103BF00008BF44EA070EB54201BFD1E905452CF4E0
:103C0000406747EA840747EA850CC3F804C0C3F855
:103C100018804F689F63C3F820E09F6947F40067EE
:103C20009F619F6927F480679F6131E00368D3F843
:103C300020C01A6A22F480522CF400541A621A46E8
:103C4000D3F804E052F81C6F8F680D6844EA073C13
:103C500026F4E64440F2004644EA052543F4806435
:103C6000C4F20106B44202BF4C692EF4804747EA11
:103C7000841EC3F804E0DD614F681F64C3F820C0F0
:103C8000DF6947F40067DF61DF6927F48067DF6180
:103C9000096909021368194300231160BDE8F04166
:103CA000002180F83C10D8B27047000010B50446DF
:103CB000002C04BF012010BD94F83D0028B900205D
:103CC00084F83C00204600F0B1F8022040F6FF32B4
:103CD00084F83D00C4F200022068016890420FDCC5
:103CE000B0F1804F1EBF40F20043C4F2000398427F
:103CF00017D040F60003C4F20003984211D014E03C
:103D000040F60043C4F2000398421EBF40F2004355
:103D1000C4F20103984204D00023C4F20103984284
:103D200003D1A36821F07001194341F6FF73C4F277
:103D3000000398420DDC90421FDCB0F1804F1EBFA3
:103D400040F20042C4F2000290423BD040F6000232
:103D500021E043F6FF72C4F20102904220DC42F2FD
:103D60000002C4F2000290421EBF0022C4F201020F
:103D7000904227D040F2004220E040F60042C4F2D8
:103D8000000290421EBF41F60002C4F200029042BF
:103D900018D041F60042C4F20002904212D015E061
:103DA00044F20002C4F2010290421EBF44F6000237
:103DB000C4F20102904205D044F20042C4F2010272
:103DC000904203D1226921F440711143E268A36952
:103DD00021F08001C262194340F200436268C4F2DC
:103DE0000103826240F480629A4204BF6269026306
:103DF000026842F004020260012242610160002078
:103E000084F8462084F83E2084F83F2084F840203F
:103E100084F8412084F8422084F8432084F8442028
:103E200084F8452084F83D2010BD00007047000054
:103E300070470000704700007047000070470000A6
:103E4000016844F600020320C4F2000202F54C436C
:103E5000994208BF0120914208BF0020032808BFF3
:103E60007047C1B2C90051FA80F040F2E851C2F285
:103E7000000101EB8000006900B1004770470000BD
:103E8000F0B581B0044620680168C268456901F058
:103E90002F0602F02003202E06D12BB1204601B0C0
:103EA000BDE8F04001F066BE5FEA017C08D005F095
:103EB000010E12F4907F8EF0010558D1002D56D0DE
:103EC0001140CA06226B3CD5012A3AD1002100914B
:103ED00001680091416800910099416911F0400F1B
:103EE00040F0D580A18DE28DE38D002B00F047815D
:103EF000891A89B209B942E1206850E8030F2268A3
:103F000020F4907042E80303002BF5D1206850E8BC
:103F1000050F226820F0010042E80503002BF5D1CF
:103F2000202084F842000020206300BF206850E871
:103F3000030F226820F0100042E80303002BF5D1A4
:103F400007E10A0640F1EA8094F84110212940F087
:103F50001681A168B1F5805F04BF2169002900F0D6
:103F60000081216A4A1C22620978416000E1CE0783
:103F700006D012F480761EBF666C46F001066664B9
:103F800001F00407012686EA97072F4302BF676CFA
:103F900047F00207676401F0020786EA57063543D7
:103FA00002BF656C45F00405656453EA0E0318BF53
:103FB0000123BCF1000F05D5012B02BF636C43F058
:103FC00008036364636C002B00F0D98011408906FC
:103FD00003D5204601F0CEFD20684169626C01F0F6
:103FE000400102F00802114307D12046FFF728FFE5
:103FF0000020606401B0F0BD206850E8030F216824
:1040000020F4907041E80302002AF5D1206850E8BE
:10401000050F216820F0010041E80502002AF5D1D2
:10402000206B01280AD100BF206850E8030F2168E7
:1040300020F0100041E80302002AF5D1202084F886
:104040004200002020632068416911F0400F02D136
:1040500073E000BF206850E8050F216820F04000A1
:1040600041E80502002AF5D1E06B002865D045F64D
:104070001921C0F600010165FEF7BCF9002800F027
:104080007E80E06B016D01B0BDE8F0400847E36B56
:1040900019684D68A28DA9B2002954D0914252D21C
:1040A000E585D969B1F5807F01D131E0206850E81C
:1040B000030F216820F4807041E80302002AF5D143
:1040C000206850E8050F216820F0010041E8050252
:1040D000002AF5D1206850E8050F216820F0400043
:1040E00041E80502002AF5D1202084F84200002092
:1040F000206300BF206850E8030F216820F0100003
:1041000041E80302002AF5D1E06BFEF731F9A28DF8
:1041100002206063E08D101A81B21CE049062ED5A2
:10412000C16821F04001C160202084F84100204690
:1041300001B0BDE8F04000F043BA204601B0BDE850
:10414000F040FFF77DBE8A4204BFD869B0F5807F9A
:1041500015D102206063204601B0BDE8F040FFF7B2
:104160006DBE216A31F8022B6FF35F22426021623B
:10417000E18C4FF6FF7201391142E18401D001B0A8
:10418000F0BDC16821F08001C160C16841F040010B
:10419000C16001B0F0BD000010B50446002C04BFA2
:1041A000012010BD94F8410028B9002084F8400097
:1041B000204600F021F8242084F841002068C168DE
:1041C00021F40051C160204601F03AFD20680169E8
:1041D00021F490410161416921F02A014161C168E6
:1041E00041F40051C16000202021606484F8411036
:1041F00084F84210606310BD2DE9F04F87B00026AF
:10420000044644F6000240F2000943F6300046F24C
:1042100028080696CDE90466CDE90266C4F20002DC
:10422000C4F20209C4F20200C4F2020821689142F9
:104230006ED041F20042C4F20102914200F0B3801C
:1042400041F20002C4F20102914240F012810027C3
:1042500002AE4FF0020A4FF0030B072501974169A8
:1042600041F010014161416901F010010191019992
:104270000197016841F002010160016801F002014B
:10428000019101990197016841F0010101603146F6
:10429000006800F00100019001988020029009F56B
:1042A0008060CDE903A7CDF814B00695FEF764FB56
:1042B0004FF400703146CDE9020A4846CDE9047B4F
:1042C0000695FEF759FB40F2001508F58C604FF09B
:1042D00000614FF48062C2F2000585E883004FF46C
:1042E0004030C5E90372C5E90577EF61C5E9080704
:1042F0002846FEF75FF9002818BFFDF787FA25204A
:1043000005210022E563AC63FEF79CFC252045E017
:104310000196016941F480210161016901F4802164
:10432000019101990196016841F00401016002A91F
:10433000006800F00400019001984FF44060029082
:104340000220CDE90306032005900720069009F519
:104350000060FEF711FB40F200454FF000604FF4A3
:104360008061C2F20005C5E900804FF40030C5E964
:104370000266C5E90416C5E90666C5E908062846C9
:10438000FEF718F9002818BFFDF740FA272005218D
:104390000022E563AC63FEF755FC2720FEF742FCE4
:1043A00007B0BDE8F08F00260196416941F0200179
:1043B0004161416901F02001019101990196016873
:1043C00041F04001016002A9006800F04000019046
:1043D00001984FF4844002900220CDE903060320A7
:1043E00005900820069009F5C050FEF7C5FA40F286
:1043F000904508F580604FF0206A4FF480694FF4D3
:104400008037C2F20005C5E9000A2846C5E9026600
:10441000C5E90496C5E90666C5E90876FEF7CAF857
:10442000002818BFFDF7F2F9E563AC6340F2405590
:1044300008F58F604021C2F20005C5E9000A05F1C8
:10444000080080E842022846C5E90566EE61C5E934
:104450000876FEF7AFF8002818BFFDF7D7F9472018
:1044600005210022A563AC63FEF7ECFB4720FEF7B5
:10447000D9FB07B0BDE8F08FB0B582B00446134653
:104480000A4694F8420020282BD1002A4FF0010060
:1044900018BF002B26D00025222045F6D12145F655
:1044A0005D3C2563A262A385656484F84200C0F682
:1044B0000001C0F6000CE06BC0E90F1C45F6252199
:1044C000C0F60001C0E9131521680431FEF724F994
:1044D00000280AD010206064202084F842000120C7
:1044E00000E00220C0B202B0B0BD019520680168B2
:1044F0000191416801910199216911B90AE000BF58
:10450000206850E8030F216840F4807041E80302FE
:10451000002AF5D1206850E8050F216840F001001D
:1045200041E80502002AF5D1206850E8050F21680E
:1045300040F0400041E80502002AF5D10020D1E713
:10454000016844F600020320C4F2000202F54C4365
:10455000994208BF0120914208BF0020032808BFEC
:104560007047C1B2C90051FA80F040F2E851C2F27E
:10457000000101EB8000C06800B1004770470000F7
:10458000016844F600020320C4F2000202F54C4325
:10459000994208BF0120914208BF0020032808BFAC
:1045A0007047C1B2C90051FA80F040F2E851C2F23E
:1045B000000101EB8000806800B1004770470000F7
:1045C000016844F600020320C4F2000202F54C43E5
:1045D000994208BF0120914208BF0020032808BF6C
:1045E0007047C1B2C90051FA80F040F2E851C2F2FE
:1045F000000101EB8000406800B1004770470000F7
:10460000FEE70000002804BF9FED150A704790EDFB
:10461000011A90ED066A90ED022A90ED077AF0EE0D
:10462000400A90ED033A90ED044A90ED055A46EEAB
:10463000410A47EE420A10EE901A21F00041B1F112
:10464000FF4F08BFF0EE400A23EE200AC0ED060A35
:1046500080ED076A06EE040A07EE050A704700BF00
:104660000000000010B50446002C08BF10BDF5EE98
:10467000C00A0020C4ED000AF1EE10FAC4E90600F9
:1046800028DD9FED201A80EE200A81EE000A04F05A
:104690000BFD9FED1D1AB7EE002ABFEE003A20EE8B
:1046A000011A20EE000A31EE024A32EE411A30EED3
:1046B000032A30EE044A30EE011A32EE022A80EE6E
:1046C000040A81EE043A82EE044A30EE001AB0EE9B
:1046D000402A09E09FED0A1AB7EE000AB0EE412A1F
:1046E000B0EE414AB0EE413A84ED014A84ED023A1F
:1046F00084ED030A84ED041A84ED052A10BD00BF81
:1047000000000000DB0F4940F304B53F002804BF60
:104710009FED1B0A704790ED033A90ED044A90ED2F
:10472000055A90ED011A90ED022AB0EE407A33EE70
:10473000046A36EE056A80EE066A16EE101A01F07B
:10474000FF41B1F1FF4F18BFB0EE467AB0EE406ABC
:1047500001EE476A02EE476A16EE101A21F0004198
:10476000B1F1FF4F08BFB0EE406A23EE060A80EDBC
:10477000066A80ED077A07EE040A07EE050A70471D
:10478000000000000146002902BFFE2040B2704731
:104790000878012832D840F23062C2F2000252F8A2
:1047A00020205AB34988A1F201210A296FD880B587
:1047B00084B0012303FA01F10B0722D111F0F00FAD
:1047C0003CD040F2FF11009108218DF8041051896E
:1047D0000B0A8DF805308DF8061091890B0A8DF8BB
:1047E00007308DF80810D1890B0A8DF809308DF843
:1047F0000A10118A0A0A8DF80B203AE0FC2040B218
:1048000070474FF40071009108218DF80410D178A1
:104810008DF8051091788DF8061051798DF80710F4
:1048200011798DF80810D1798DF8091091798DF8EA
:104830000A10517A8DF80B10117A1AE040F2FF211C
:10484000009108218DF80410518A0B0A8DF805306B
:104850008DF80610918A0B0A8DF807308DF8081034
:10486000D18A0A0A8DF809208DF80A1000218DF8E6
:104870000B108DF80C106946FCF7AEFA002818BF33
:104880004FF0FF3004B0BDE8804040B27047FF20D9
:1048900040B2704710B500B3017801291DD840F22D
:1048A0003062C2F2000252F8211000291CBF91F8B8
:1048B00044E0BEF1000F10D001F1180C002300BF3E
:1048C0005CF8231019B142884C88944203D001331C
:1048D0007345F5DB0021084610BD0021084610BDD8
:1048E000F0B581B0044624B12678012E05D9FF2009
:1048F00000E0FE2040B201B0F0BD40F23067C2F2ED
:10490000000757F82600B8B157F8266036B396F876
:10491000440028B306F11801002200BF51F82230EC
:104920001BB167885B88BB4238D001328242F5DB1D
:104930000A2815D9FF20DDE74820FCF7E1FA0546F3
:10494000002D47F8265027D028464821FBF795FC34
:104950002E702678012ED7D9FF20CBE7FF20C9E79C
:104960005020FCF7CDFA0546D5B120686168696032
:10497000286005F118002821FBF77FFC60790322ED
:1049800085F8280061882078FBF74CFF50B1284655
:10499000FCF7B4FAFF20ADE7FF20ABE7FD20A9E765
:1049A000FF20A7E796F8440006EB8000856196F8A3
:1049B0004400013086F8440000209BE710B5002831
:1049C00002BFFE2040B210BD0178012934D840F268
:1049D0003062C2F2000252F821C0BCF1000F2BD0AD
:1049E000B7EE001ABFEE002AB4EEC10AF1EE10FADB
:1049F000C8BFB0EE410A41799CF844E0B4EEC20A67
:104A0000F1EE10FAB8BFB0EE420AB1EE401A00293A
:104A100008BFB0EE401ABEF1000F0DD00CF1180126
:104A2000002200BF51F822301BB15B884488A342AA
:104A300005D001327245F5DBFC2040B210BD007993
:104A4000022805D2A3F2012189B2072906D31EE06C
:104A50001DD1A3F2052189B2052918D849F2EC31FC
:104A600040B2C0F6000101EB800090ED000A4FF06B
:104A70007F4000EB03600CEBE05021EE000ABDEE3E
:104A8000C00A10EE101A4180002040B210BDFF2075
:104A900040B210BDF0B587B0024622B110780128AF
:104AA00003D9FC201DE0FE201BE040F23061C2F281
:104AB000000151F8201089B191F8443083B101F11F
:104AC0001804002554F825701FB179885688B14222
:104AD0000AD001359D42F5DBFC2002E0FC2000E01D
:104AE000FC2040B207B0F0BD6A460023FBF7D0FDC2
:104AF00078B1FCF707FAD7E90823801A40F2E932C7
:104B00009941801A71F1000028D300203876FC20EA
:104B1000E7E701203876FCF7F5F9C7E908019DF8C9
:104B200011009DF8121097F904509DF80E309DF871
:104B30000F209DF8106041EA00219DF80D0046EA23
:104B40000222022D43EA00200AD84FA64BA306EB0F
:104B5000850653F8253096ED004A05E0FF20C0E7B2
:104B6000B7EE004A4FF0FF339FED4A1A09B200EE4C
:104B7000100A12B29FED483A5943B8EEC05A06EEF9
:104B8000102A9FED460A02EE101AB8EEC22A25EE50
:104B9000015AB8EEC61AB97922EE032A25EE003A78
:104BA00041B1B7F84010411AB1F5805F08DD4FF010
:104BB000FF3109E000217964A7F84000B96418E0EA
:104BC00011F5805F04DA01217A6C1144796400E008
:104BD000796C05EE101A81EE041A24EE022AB8EE62
:104BE000C55AA7F8400005EE003A83EE043A87ED77
:104BF000123A87ED023A87ED031A87ED042A97F8F7
:104C0000280048B3B5EEC03AF1EE10FA08DA33EEF8
:104C1000003AB5EEC03AF1EE10FAF8DB87ED023A51
:104C2000B4EEC03AF1EE10FA0ADB9FED1D4A33EE06
:104C3000043AB4EEC03AF1EE10FAF8DA87ED023A2F
:104C400030EE430AB1EE411AB1EE422A87ED020A74
:104C500087ED031A87ED042A9DF8130007F1080376
:104C600007F12C0C00EE100AB8EE400A87ED050A99
:104C70000FCB8CE80F00002033E700BF10270000A7
:104C80000040000030750000000010420000984114
:104C90000000803F0000003900008038DB0FC94071
:104CA000DB0FC9C080B540F62C1046F200414FF42E
:104CB0001022C2F20000C4F2000101600321416031
:104CC0000021C0E9021102614FF4001242618183A8
:104CD0008161FDF77BF800281CBFBDE88040FCF730
:104CE00095BD80BD80B540F6541046F600014FF4E6
:104CF000C022C2F20000C4F2000101600321416041
:104D00000021C0E9021102614FF4A00242618183D7
:104D10008161FDF75BF800281CBFBDE88040FCF70F
:104D200075BD80BD80B582B043F630010020019092
:104D3000C4F202010A6842F400120A600A6802F42E
:104D400000120192019A00900868002240F480004D
:104D500008600868052100F48000009000980C208D
:104D6000FDF770FF0C20FDF75DFF392005210022C3
:104D7000FDF768FF3920FDF755FF3A200521002295
:104D8000FDF760FF3A20FDF74DFF3B200521002293
:104D9000FDF758FF3B20FDF745FF44200521002289
:104DA000FDF750FF4420FDF73DFF4520052100227F
:104DB000FDF748FF452002B0BDE88040FDF732BF57
:104DC00080B545F2657049F284420021C0F60000CA
:104DD000C0F6000201F04CFB40F6281149F21042E7
:104DE000C2F20001C0F60002086045F6550000213D
:104DF000C0F60000BDE8804001F03ABB2DE9F04765
:104E000086B043F630000026002400224FF4E05A1A
:104E100005960096C4F20200C4F20204016804F58B
:104E2000E05741F002010160016801F002010091C8
:104E300000990096016841F040010160016801F0AD
:104E40004001009100990096016841F00101016064
:104E5000016801F00101009100990096016841F09C
:104E600008010160016801F00801009100990096B5
:104E7000016841F004010160016801F00401009142
:104E800000990096016841F080010160016801F01D
:104E90008001009100990096016841F020010160B5
:104EA0004FF4E051006800F0200000900098384670
:104EB000FDF742FE2046102101224FF01009012586
:104EC000FDF73AFE04F58068012101224046FDF716
:104ED00033FECDE901A50396022001AE04903846C9
:104EE0003146FDF749FD4FF48817204631460195BC
:104EF000CDE90275FDF740FD20463146CDE901952B
:104F0000CDE90355FDF738FD30203146CDE90107E5
:104F100004F500600395FDF72FFD40463146CDE9CD
:104F20000155CDE90355FDF727FD06200521002297
:104F3000FDF788FE0620FDF775FE0A2005210022F8
:104F4000FDF780FE0A20FDF76DFE172005210022E7
:104F5000FDF778FE1720FDF765FE06B0BDE8F08787
:104F600010B540F67C1043F200014FF4827200232A
:104F70004FF0010C4FF4007E1824C2F20000C4F27E
:104F8000010180E80E000A21C0E90333C0E905CE23
:104F9000C461C0E90833C0E90A31FEF791F900287D
:104FA0001CBFBDE81040FCF731BC10BD70B58EB021
:104FB00040F6D41044F20045002141F28732C2F29B
:104FC0000000C4F201050791CDE90511CDE90311F7
:104FD000CDE90111C0E90051C0E90212016181610E
:104FE000FEF7E2FA002818BFFCF710FC40F6D410D8
:104FF000C2F20000FEF75AFE002818BFFCF706FCBC
:1050000040F6D4146020002601A90022C2F2000458
:105010000190CDE9026605962046FEF731FD002895
:1050200018BFFCF7F3FB0D96CDE90B66CDE90966D9
:1050300043F630002168C4F20200A9421FD040F6B6
:105040000002C4F20002914231D1002108910268AD
:1050500042F008020260006800F00800089008981A
:105060004FF4804009900220CDE90A01CDE90C10EF
:1050700005F5484009A9FDF77FFC0EB070BD002181
:105080000891026842F020020260006800F02000EF
:1050900008900898402009900220CDE90A010C9060
:1050A000032009A90D9005F55040FDF765FC0EB0F1
:1050B00070BD0000B0B594B040F61C2040F600056D
:1050C000002145F20722C2F20000C4F200050D9152
:1050D000CDE90B11CDE90911CDE90711CDE9051194
:1050E000CDE90311CDE90111C0E90051C0E9021277
:1050F00001618161FEF758FA002818BFFCF786FBB2
:105100004FF480500AA90A9040F61C20C2F2000019
:10511000FEF754FB002818BFFCF778FB40F61C2074
:10512000C2F20000FEF7C2FD002818BFFCF76EFBBC
:1051300040F61C20002408A9C2F20000CDE9084472
:10514000FEF7D4F9002818BFFCF760FB602001A926
:105150000822CDE901040394059440F61C24C2F210
:1051600000042046FEF78CFC002818BFFCF74EFB1D
:10517000002044F2004343F630011390CDE91100C2
:10518000CDE90F00C4F20103C4F2020122689A4281
:105190001BD0AA4230D100200E900A6842F00802CB
:1051A0000A60096801F008010E910E994FF48041E0
:1051B0000F910221CDE91010CDE9120105F5013062
:1051C0000FA9FDF7D9FB14B0B0BD0E900A6842F0EC
:1051D00020020A60096801F020010E910E99402119
:1051E0000F910221CDE91010032012910FA9139005
:1051F00005F50330FDF7C0FB14B0B0BD10B582B0AB
:1052000040F6642041F20041002440F2473240F26F
:10521000E733C2F20000C4F20001CDE9004480E8A7
:105220001600C3608461FEF7BFF9002818BFFCF7C1
:10523000EDFA40F664206946CDE90044C2F2000070
:10524000FEF754F9002818BFFCF7E0FA02B010BDD1
:1052500080B540F6AC2041F200014FF4E13200236A
:105260004FF00C0CC2F20000C4F2010180E80E0005
:10527000C0E90333C0E905C3C361FEF78DFF002811
:105280001CBFBDE88040FCF7C1BA80BD80B540F6C8
:10529000F42044F6000C48F2A0624FF48053002141
:1052A0004FF00C0EC2F20000C4F2000CC0F201027A
:1052B000C0E900C2C0E90231C0E9041EC0E906111C
:1052C000FEF76AFF00281CBFBDE88040FCF79EBACD
:1052D00080BD000080B540F63C3041F200414FF403
:1052E000E13200234FF00C0CC2F20000C4F20101C5
:1052F00080E80E00C0E90333C0E905C3C361FEF7CF
:105300004BFF00281CBFBDE88040FCF77FBA80BD82
:10531000FEE70000F0B581B02DED048BB0EE408AC1
:105320001446A8B10078052816D8DFE800F01985E2
:10533000990303A5012B0DDB00200022002100BFF3
:10534000013144F82200CAB29342F9DCFF206EE03A
:10535000FF206CE0FF206AE0012B35DA002066E0D8
:10536000042BE7D191ED000A91ED011A91ED022A8B
:1053700030EE410A30EE020A84ED000A91ED000A97
:1053800091ED011A91ED022A30EE010A30EE020A87
:1053900084ED010A91ED000A91ED011A91ED022AC6
:1053A00031EE400A30EE020A84ED020A91ED000A65
:1053B00091ED011A91ED022AB1EE400A30EE410A58
:1053C00030EE020A84ED030A9FED2E9ADDB22746E5
:1053D0002E4600BF97ED000A03F0CBFCB4EEC90ADD
:1053E000013E0437F1EE10FAC8BFB0EE409A002E2D
:1053F000F0D1B7EE000AB4EEC09AF1EE10FA0BDD70
:105400002846214691ED000A013880EE090A81ED17
:10541000000A01F10401F5D194ED000A013D20EEEE
:10542000080A84ED000A04F10404F5D1002040B21A
:10543000BDEC048B01B0F0BD042B7FF47BAF91ED8C
:10544000000AB1EE400A84ED000A0868606008684E
:10545000A06091ED000AB1EE400A84ED030A6BE70B
:10546000022B7FF467AF91ED000AB1EE400A84EDA4
:10547000000A086860605FE7012B7FF45BAF086893
:10548000206059E70000000000280EBFFF200170D7
:10549000002040B270470000FEE70000B0B52DEDDF
:1054A0000A8B044610EE100AB0EE618AB0EE419A03
:1054B000B0EE60BA00F0FF40B0F1FF4F00F09B800B
:1054C0001BEE100A00F0FF40B0F1FF4F00F0938098
:1054D00019EE100A00F0FF40B0F1FF4F00F08B8092
:1054E00018EE100A00F0FF40B0F1FF4F00F083808B
:1054F0006068F0EE4B0A90ED071AFBF7FDFF60685D
:10550000B0EE40AA90ED001A04F11C0021EE0B0A47
:105510002AEE01CAFFF776F82078B0EE40BA70B1F3
:1055200001280ED194ED050AD4ED020A3BEE409A13
:10553000B0EE480A03F0CCFC89EE009A01E09FED42
:10554000309A84ED04AA84ED05BA19EE100A9FED95
:105550002C0A656894ED03AA00F0FF40B0F1FF4FFC
:105560000CEE08AA95ED022A9FED268A95ED011A08
:1055700095ED033A18BFB0EE490A2CEE019AB4EE4D
:10558000C82A2AEE02BA00EE439AF1EE10FA1EDDA6
:105590001AEE100A00F0FF40B0F1FF4F17D039EEBD
:1055A0000B0A03F0E6FB95ED051AB4EEC10AF1EE25
:1055B00010FA0CDCB0EE4A0A03F0DBFB95ED041A9E
:1055C000B4EEC10AF1EE10FAD8BF84ED03AA39EEA9
:1055D0000B0A10EE100A00F0FF40B0F1FF4F0AD0A6
:1055E000D5ED050AF4EEC80AF1EE10FAC8BFFBF7D4
:1055F00037F884ED060A94ED060ABDEC0A8BB0BDBF
:1056000000000000BD37863570B504460D464CB32A
:10561000506800F0FF40B0F1FF4F23D0906800F0D9
:10562000FF40B0F1FF4F1DD0D06800F0FF40B0F157
:10563000FF4F17D0106900F0FF40B0F1FF4F11D0BD
:10564000506900F0FF40B0F1FF4F0BD0B7EE001AE9
:10565000626081EE001A11EE100A00F0FF40B0F116
:10566000FF4F02D1FF2568B270BD84ED021A04F12C
:105670001C06D2ED060A3046FEF7F4FF9FED060A3F
:10568000257000253046C4E90355C4E90555FFF7E8
:105690003DF868B270BD00BF0000000010B50028E2
:1056A00002BFFF2460B210BD9FED050A0024C0E9CF
:1056B0000344C0E905441C30FFF728F860B210BD70
:1056C00000000000000000000000000000000000DA
:1056D000EFF30980BFF36F8F154B1A681EF0100FA0
:1056E00008BF20ED108A20E9F04F10602DE9090075
:1056F0004FF0500080F31188BFF34F8FBFF36F8FCF
:1057000002F0F2F84FF0000080F31188BDE80900C4
:1057100019680868B0E8F04F1EF0100F08BFB0EC31
:10572000108A80F30988BFF36F8F704700BF00BFF6
:10573000240C002000000000000000000000000019
:10574000074B19680868B0E8F04F80F30988BFF389
:105750006F8F4FF0000080F31188704700BF00BFCB
:10576000240C002080B500F081FEBDE8804000F0F0
:10577000CFBE000080B5FDF7EBF903F011F801286A
:105780001CBFBDE8804002F087B980BDB0B592B0C3
:1057900043F6400000240225CDE90A44CDE908443F
:1057A0000594CDE90344CDE901440094C4F202001C
:1057B000016841F080510160006800F08050009065
:1057C0000098009447F20000C4F20000016841F420
:1057D00080410160006800F4804000900098012042
:1057E00006904FF4803007904FF480000C950D9098
:1057F00006200E90A820CDE90F050420119006A8E0
:10580000FDF772FB08B172B6FEE70F200521CDE966
:1058100001054FF4A050039404904FF4805005907C
:1058200001A8FDF751FA002804BF12B0B0BD72B64E
:10583000FEE700004EF68850CEF20000016841F409
:10584000700101607047000040F66420C2F2000061
:10585000FEF786B810B500F0B3FB45F6D90049F263
:1058600034420021C0F60000C0F6000200F000FE45
:1058700041F2880449F258420021C2F20004C0F605
:105880000002206045F66910C0F6000000F0F0FD4F
:10589000606002200A21002200F02AFCA0600220A1
:1058A0005821002200F024FCE06002201021002298
:1058B00000F01EFC606102200421002200F018FCB0
:1058C000A06100F0B3FB00F0D1FDBDE8104000F096
:1058D0001FBE000000000000F0B581B000F056FBD4
:1058E0000646002000F01EFB00F048FB0546FBF7D3
:1058F00035FE9FED1B0A40F238640146C2F20004F7
:105900002046FBF705FD3046FAF790FD9FED120BA0
:1059100053EC102BFAF7BCFC42F6F602C4F28402F8
:105920002263FAF790FD40F6181706463544C2F296
:10593000000700BF2046FBF7AFFD00F01FFB02464B
:1059400020463946FBF760FB2046FBF779FD2846E9
:1059500000F0F8FA3544EDE70000000000407F4019
:105960000000FA43000000002DE9F04700F00EFBB4
:105970000446002000F0D6FA2046FAF757FD9FEDC6
:10598000240B53EC102BFAF783FCFAF75CFD04466A
:1059900000F0F4FA40F230364FF6F87841F2880A17
:1059A00005194FF40139C2F20006C0F2FF08C2F235
:1059B000000A06F110070AE0DAF814003146002266
:1059C000002300F0D5FB284600F0BCFA25443846F9
:1059D000FBF7F2FE1420FBF7FFFE012814D1384636
:1059E000FBF7F4FD96F84900411E002002299CBFF8
:1059F00008EAC10029FA00F03070B06B7060706B7B
:105A0000B060F06BF060D7E73846FBF7D1FDD3E725
:105A10000000000000407F40806B0021C185FEF740
:105A20000FBA0000806B01684A6990F84130212B61
:105A300014D112F0800211D00022C28401E000BF14
:105A4000016851E8031F026821F0C00142E8031316
:105A5000002BF5D1202180F8411001684A6990F8A7
:105A60004230222B2DD112F040022AD00022C285D2
:105A700001E000BF016851E8031F026821F4907142
:105A800042E80313002BF5D1016851E8051F0268B5
:105A900021F0010142E80513002BF5D1016B01292A
:105AA0000AD100BF016851E8031F026821F010010C
:105AB00042E80313002BF5D1202180F84210002189
:105AC0000163416C41F010014164FEF7B9B9000077
:105AD0000168806B096811F4807F32D10021C18593
:105AE000016851E8031F026821F4807142E8031342
:105AF000002BF5D1016851E8051F026821F0010172
:105B000042E80513002BF5D1016851E8051F026832
:105B100021F0400142E80513002BF5D120218446F5
:105B200080F842105CF8302F012A0CD1026852E84C
:105B3000032F036822F0100243E803210029F5D166
:105B400001E000F1300C00214163DCF80010012974
:105B500018BFFEF7F5BC818DFEF770B9806B01218F
:105B60004163016B012918BFFEF70ABD818D490809
:105B7000FEF764B990F84210222918BF7047836875
:105B8000B3F5805F06D1026900F12801A2B1D1F816
:105B900000C008E00146002B51F828CF01D103696D
:105BA0000BB17F2300E0FF23026852681A400123F3
:105BB0008CF800200A6806E00368826A5B686FF36D
:105BC0005F23138002231A440A604FF6FF72C18DCF
:105BD00001391142C18500D070470168CA6822F0BE
:105BE0002002CA60CA6822F48072CA604A6922F040
:105BF00001024A61202280F8422000224263036BA6
:105C0000012B18BFFEF79CBC026300BF51E8031FC5
:105C1000026821F0100142E803130168002BF5D15E
:105C20000A6812F0100F08D081B0002200920A68B2
:105C3000009249680091009901B0818DFEF7FEB88D
:105C4000B0B5044649F20C6520680169E26821F4A8
:105C5000405111430161D4F808C0D4E90423D4F8B9
:105C60001CE0C16842EA0C02A9431A4342EA0E0250
:105C70001143C1604169A26921F44071114341613E
:105C800041F2004140F48060C4F20101884202D137
:105C9000FDF7E0F801E0FDF7C9F8E2696368192152
:105CA000A0FB0101B2F5004F1CD15A00DB0FFAF73F
:105CB00087FA48F21F51C5F2EB11A0FB01235A09E4
:105CC0006FF0630302FB0300322303EBC000A0FB71
:105CD00001014FF4F87000EA1110C1F3421100EB1A
:105CE00002101AE09A009B0FFAF76AFA48F21F5165
:105CF000C5F2EB11A0FB01235A096FF0630302FB0D
:105D00000300322303EB0010A0FB0101F02000EAA6
:105D10005110C1F3431100EB021008432168886061
:105D2000B0BD000040F6AC20C2F20000FEF7A8B8FB
:105D300010B582B040F6F420C2F20000006801689D
:105D400011F0200F3BD144F60001C4F200010968B4
:105D500011F0100F55D0002141F2C8030091C2F29A
:105D600000030168009140680090009840F20040F4
:105D7000C2F2000000680268016821F0010112F41B
:105D8000002F01604168C1F1320119804FF03203E8
:105D900043601DD1026842F400220260026842F0B2
:105DA0000102026088B219282BD140F2D020C2F241
:105DB0000000283002B0BDE8104001F02DB80021ED
:105DC00001910168019140680190019802B010BDF5
:105DD00046F22802C4F20202136823F4002313607F
:105DE000026842F00102026088B2192809D140F22B
:105DF000D024C2F2000404F1410001F00DF80120AA
:105E0000207002B010BD000010B540F63C34C2F264
:105E100000042046FEF734F82046BDE81040FBF7AA
:105E2000A9B80000FEE700002DE9F04104466CB37C
:105E300040F62440C2F200000068A04202BF0020E9
:105E4000C0B2BDE8F08101F099F940F260186569CF
:105E5000C2F20008D8F81860D8F81C7001F0B4F944
:105E6000B5424FF0020018BFBD420CD008F14C0003
:105E7000854214D00120002D08F1380108BF04200C
:105E80008D4208BF0420C0B2BDE8F0814FF0500041
:105E900080F31188BFF36F8FBFF34F8FFEE7A06AC7
:105EA00000281EBF0220C0B2BDE8F08194F858104F
:105EB0000320012908BF0220C0B2BDE8F081000024
:105EC00080B5FCF74FFEFFF761FCFEF797FFFEF78A
:105ED00029FFFEF7E7FEFEF705FFFFF7D7F9FFF70B
:105EE000F9F9FFF73DF8FFF7B3F9FFF7E3F8FFF72C
:105EF00085F9FFF75BF800F04DF8FEF761FF00F061
:105F000075F800BFFEE7000032EE612A30EE600A4D
:105F100031EE601A20EE020A80EE010A30EE210A0C
:105F200070470000EFF3058100291CBF6FF00500EA
:105F30007047002804BF0020704780B501F05CFA6C
:105F4000002080BD10B582B00446EFF30580002824
:105F50001EBF6FF0050002B010BD02F031FC211A27
:105F600001900129BEBF6FF0030002B010BD01A86F
:105F700001F08CFA002002B010BD0000EFF30580A4
:105F8000002808BF02F01CBC02F020BC4FF47A705D
:105F900070470000EFF3058000281CBF6FF005007C
:105FA000704740F2E450C2F20000016800291CBFB3
:105FB0004FF0FF3070470121016000207047000062
:105FC00080B5EFF3058010B16FF0050080BD02F0E1
:105FD000E7FB002804BF012080BD02281CBF4FF052
:105FE000FF3080BD01F078FC002080BD10B5EFF3DC
:105FF000058000281EBF6FF00504204610BD40F24A
:10600000E450C2F20000016801291EBF4FF0FF34C6
:10601000204610BD4EF61F510024CEF200010C7038
:106020000221016001F012FC204610BD10B5EFF313
:10603000058000281EBF6FF00504204610BD02F049
:10604000AFFB022802BF0024204610BD60B902F059
:10605000A7FD0124012809D002F0A2FB002808BFF7
:106060004FF0FF34204610BD4FF0FF34204610BDE6
:1060700010B582B0B1FA81F21C46B0FA80F3520931
:106080005B091A43EFF30583EBB1002C18BF012421
:10609000224319D10022019201AA02F0F1F801284D
:1060A0001EBF6FF0020002B010BD0198A8B14EF6FD
:1060B00004504FF08051CEF200000160BFF34F8FCB
:1060C000BFF36F8F09E01AB16FF0030002B010BD8B
:1060D000224602F007F8012802D1002002B010BDCC
:1060E0006FF00100002C08BF6FF0020002B010BD7D
:1060F000B0B582B000291446EFF305824FF00005D9
:1061000018BF002830D07ABB04B3D4E9023273B18F
:10611000502A0FD322699AB1D4F814E001FB00FC95
:106120000025E64520D3009501F09EFD11E01AB14F
:10613000002519E0002517E022691AB1002513E0B7
:10614000002511E062690AB100250DE0002201F08E
:1061500045FD05463DB1002C284614BF21680021AD
:1061600001F0ECF800E00025284602B0B0BD0000C8
:10617000B0B582B0B1FA81F21D46B0FA80F352098F
:106180005B091A43EFF305833BB1002D18BF0125CE
:106190002A4306D06FF003042CE0CAB16FF0030469
:1061A00028E000220023019201AA01F0D3FE012879
:1061B0001CD10198E8B14EF604504FF080510024F4
:1061C000CEF200000160BFF34F8FBFF36F8F11E07D
:1061D0002A460023002401F0B7FD01280AD06FF001
:1061E0000104002D08BF6FF0020403E06FF0020409
:1061F00000E00024204602B0B0BD000010B50C46FF
:106200000146EFF3058010B16FF0050010BD21F0DD
:106210000100002804BF6FF0030010BD11F0010160
:1062200007D1214602F088F8012804BF002010BDE4
:1062300006E0214602F062F9012804BF002010BDEB
:106240006FF00100002C08BF6FF0020010BD0000CD
:1062500070B50446EFF3058010B10025284670BDE7
:1062600094B1606810F0080FF7D100F00106D4E98E
:10627000021031B15028F0D3D6B9012001F05CFCF6
:1062800005E00028E9D1DEB9012001F01DFC05463A
:106290000026002DE1D0002C284614BF21680021E3
:1062A00001F04CF8002E18BF45F00105284670BDDE
:1062B000042001F041FC05460126002DEBD1CCE77E
:1062C000042001F001FC0546002DE4D1C5E70000E3
:1062D00080B50146EFF3058000281CBF6FF0050074
:1062E00080BD21F00100002804BF6FF0030080BDD5
:1062F00011F001010BD100210022002301F024FD47
:106300006FF00201012808BF0021084680BD01F09E
:10631000C7FE01466FF00200012908BF002080BDC2
:106320002DE9F04F81B08146EFF3058017460C460A
:1063300028B16FF0050B584601B0BDE8F08FB9F1F8
:10634000000F15DB14F0020F4E466FF0010B18BF63
:106350000026002F08BF6FF0020B02F031FA8046D2
:1063600014F0010F07D1002F47D00025EA4619E0AD
:106370006FF0030BDFE7002F5AD00024EA4625E038
:1063800002F01EFAA0EB08003F1A38BF002709E010
:10639000009904EA090041EA000515EA090FEFD067
:1063A00061E000BF0020314652463B462C4602F0D9
:1063B000A7FA0028BFD001285D46F3D1E8E702F034
:1063C000FFF9A0EB08003F1A38BF00270020314634
:1063D00052463B46254602F093FA0028ABD00128EE
:1063E0005C46F3D1009905EA090041EA000404EA99
:1063F00009004845E3D1A3469DE700206C4600BF55
:106400000546002031462246002302F079FA002892
:106410003FF491AF01285846F2D1009905EA0900EE
:1064200041EA000B1BEA090F08BF6FF0020B82E77D
:1064300000206C460546002031462246002302F02B
:106440005FFA00283FF477AF01285846F2D100994F
:1064500005EA090041EA000B0BEA0900484518BFAC
:106460006FF0020B67E7AB4665E7000002F092B9F8
:10647000F0B585B000238C4600280493EFF3058126
:106480003BD0D1BB42B19469002C08BF1824611ED7
:10649000372911D9002330E000218023182404AAD1
:1064A000CDE900429AB2634602F08CF801281ABF87
:1064B00000230493049B20E01179C9071CD11168C3
:1064C000D2E9025756694FEA960E002E734608BF6E
:1064D0008023ADB100235C2F0FD3002E1CBF1269A7
:1064E000002A0AD0CDE9004272466346029502F0C6
:1064F000D7F80346049300E00023184605B0F0BD2A
:106500000FB10023F9E71269002AC8D00023F4E78D
:1065100010B50446EFF3058000281CBF6FF005009E
:1065200010BD64B12046FFF77FFC042804BF6FF064
:10653000020010BD204601F01BF8002010BD6FF0D6
:10654000030010BD2DE9F041044600F017FE40F2B3
:10655000601740F62448C2F20007C2F20008B8688B
:106560000130B860D8F8000060B1F868002840F049
:106570000C81D8F80000E16AC06A884298BFC8F868
:10658000004002E1C8F80040B868012840F0FD80F2
:1065900040F62845C2F20005284600F0ABFD05F1A3
:1065A000140000F0A7FD05F1280000F0A3FD05F19F
:1065B0003C0000F09FFD05F1500000F09BFD05F14F
:1065C000640000F097FD05F1780000F093FD05F1FF
:1065D0008C0000F08FFD05F1A00000F08BFD05F1AF
:1065E000B40000F087FD05F1C80000F083FD05F15F
:1065F000DC0000F07FFD05F1F00000F07BFD05F50B
:10660000827000F077FD05F58C7000F073FD05F5E4
:10661000967000F06FFD05F5A07000F06BFD05F5BC
:10662000AA7000F067FD05F5B47000F063FD05F594
:10663000BE7000F05FFD05F5C87000F05BFD05F56C
:10664000D27000F057FD05F5DC7000F053FD05F544
:10665000E67000F04FFD05F5F07000F04BFD05F51C
:10666000FA7000F047FD05F5027000F043FD05F5F6
:10667000077000F03FFD05F50C7000F03BFD05F5DF
:10668000117000F037FD05F5167000F033FD05F5CB
:106690001B7000F02FFD05F5207000F02BFD05F5B7
:1066A000257000F027FD05F52A7000F023FD05F5A3
:1066B0002F7000F01FFD05F5347000F01BFD05F58F
:1066C000397000F017FD05F53E7000F013FD05F57B
:1066D000437000F00FFD05F5487000F00BFD05F567
:1066E0004D7000F007FD05F5527000F003FD05F553
:1066F000577000F0FFFC05F55C7000F0FBFC05F541
:10670000617000F0F7FC05F5667000F0F3FC05F52C
:106710006B7000F0EFFC05F5707000F0EBFC05F518
:10672000757000F0E7FC05F57A7000F0E3FC05F504
:106730007F7000F0DFFC05F5826000F0DBFC05F205
:10674000244000F0D7FC05F5876000F0D3FC05F28B
:106750004C4000F0CFFC40F26045C2F200052846F4
:1067600000F0C8FC05F11406304600F0C3FC07F148
:10677000600000F0BFFC07F1380000F0BBFC07F13F
:106780004C0000F0B7FCBD61FE6138680130386034
:106790006064E06A396A884240F6284188BF3862FE
:1067A00000EB8000C2F2000101EB8000211D00F02F
:1067B000CFFC00F009FDF86890B1D8F80000E16A5C
:1067C000C06A884228BFBDE8F0814EF604504FF001
:1067D0008051CEF200000160BFF34F8FBFF36F8F87
:1067E000BDE8F0812DE9F04140F2601540F6284601
:1067F0004EF604584FF08057C2F20005C2F2000670
:10680000CEF2000803E000BF204600F0F5FC686807
:10681000D0B100F0B3FC686CC468201D00F03CFCF3
:10682000A8680138A86068680138686000F0CCFC8E
:1068300094F8590020B10128E6D00228E7D00DE0F5
:10684000206B00F0D9FCDFE730680228DFD3C8F8FE
:106850000070BFF34F8FBFF36F8FD8E74FF050003A
:1068600080F31188BFF36F8FBFF34F8FFEE70000F7
:1068700008480068006880F308884FF0000080F343
:10688000148862B661B6BFF34F8FBFF36F8F00DF1E
:1068900000BF00BF08ED00E02DE9F04F85B0814654
:1068A00001F08EFF40F2E0148346C2F2000420693A
:1068B000834538D2A068016881B34FF0000A0DF11A
:1068C000040800BFC068C76805683E1D304600F078
:1068D000E3FB396A3846884797F82800400719D5FE
:1068E000B8692844A84207D978603F613146A0685A
:1068F00000F010FC0EE000BF2068E8B1CDE901A572
:10690000039701F04DFF206841460022002301F06B
:106910001BFA88B1A06801680029D3D1E168C4E9F5
:106920000210012000E00020C9F80000C4F810B0F7
:10693000584605B0BDE8F08F4FF0500080F3118845
:10694000BFF36F8FBFF34F8FFEE7000081B00020D1
:10695000009040F29800C2F2000000684FF0500131
:1069600081F31188BFF36F8FBFF34F8F013001D0D8
:10697000FEE700BF00980028FCD001B0704700007F
:106980002DE9F04F89B040F2E01601AC4FF000095C
:106990000DF11408EA46C2F2000600BFB0684FF0DD
:1069A000000B0768002F1CBFC068D0F800B000F0D3
:1069B00093FF2046FFF770FF0546019810B102F0E3
:1069C000EFF84DE0AFB15D4513D302F0E9F8B068E0
:1069D000C068C76807F10409484600F05DFB97F8F6
:1069E000280010F0040F1FD100F0FE0087F82800E7
:1069F0002CE0002227B9F0680068B0FA80F0420964
:106A00003068ABEB050100F0D3FC02F0C9F838BBED
:106A10004EF604504FF08051CEF200000160BFF3FB
:106A20004F8FBFF36F8F1BE0B86900EB0B01A942DA
:106A300079603F6101D9B06805E0A5EB0B018142A7
:106A400080F08C80F068494600F064FB4FF000094C
:106A5000396A3846884703E000F0FE0087F82800CE
:106A600030682146002201F03DFB002896D00198B5
:106A7000B0F1FF3F06DCDDE9022004999047019860
:106A80000028EDDB039F786900281CBF381D00F04B
:106A900003FB5046FFF700FF01990929E0D8DFE822
:106AA00001F0050505373A530505373A97F82810E0
:106AB00041F0010187F82810391DBD69029AAB1811
:106AC00083427B603F6104D9904235D2934203D226
:106AD00032E0801AA84233D3396A3846884797F89B
:106AE00028004007BCD53268B8690299002A50D006
:106AF0000844CDF81490CDE9060701F051FE306846
:106B000041460022002301F01FF90028A8D140E0EF
:106B100097F82800A0E797F8281041F0010187F8BE
:106B2000281002990029B9613DD00A18394641F868
:106B3000042F82423F6103D9B06800F0EBFA8FE77F
:106B4000F06800F0E7FA8BE797F8280010F0020FE2
:106B50007FF482AF384600F04FFB81E7306878B1B0
:106B60004FF00009CDE9059B079701F019FE306849
:106B700041460022002301F0E7F800287FF468AFC7
:106B80004FF0500080F31188BFF36F8FBFF34F8F2A
:106B9000FEE74FF0500080F31188BFF36F8FBFF313
:106BA0004F8F00BFFEE74FF0500080F31188BFF316
:106BB0006F8FBFF34F8F00BFFEE70000F0B581B0CD
:106BC000044600F0DBFA94F94560012E10DB04F175
:106BD000240500BF286858B1284601F09FFF00280F
:106BE00018BF00F043FD71B2701E01290646F1DCAA
:106BF000FF2684F8456000F0E7FA00F0BFFA94F948
:106C00004470012F10DB04F1100500BF286858B153
:106C1000284601F083FF002818BF00F027FD79B255
:106C2000781E01290746F1DC84F8446001B0BDE814
:106C3000F04000F0C9BA000070B5044600F04CFE08
:106C400040F22020C2F20000016849B145F69431BB
:106C5000C2F200010978002918BF4FF000412AE074
:106C600041F6DC060025C2F20006F31D16F007020D
:106C7000314623F0070318BF19469B1B4FF470568B
:106C8000002AC0E9051518BFC3F570568A19083ADD
:106C900022F007020260C2E90055521A4A600368F6
:106CA0000B6045F69431C0E901220122C2F20001D5
:106CB0000A704FF000410025002C00F07D8021403B
:106CC0007AD104F1080313F007010ED0C1F10801D5
:106CD0000B4413F0070F08D04FF0500080F31188D9
:106CE000BFF36F8FBFF34F8FFEE741685A1E8A4292
:106CF00021D2064656F8142F3146164675689D4235
:106D000002D23268002AF7D10268964213D0326864
:106D1000D1F800E00A60E91A112933D3F51815F00B
:106D2000070F0AD04FF0500080F31188BFF36F8F28
:106D3000BFF34F8FFEE700253EE06960736000F10E
:106D4000140300BF1C462368AB42FBD36168621882
:106D5000AA4202D0D5F804C005E06A68254602EBD5
:106D6000010CC4F804C005EB0C01994206D101687E
:106D70008B421FBF5968614469601B68AC422B603D
:106D800018BF2560716842680EF10805521A42600A
:106D900083689A4238BF826045F69432C2F200029C
:106DA0001278002A4FF0000218BF41F00041C6E9F6
:106DB0000021C1680131C16001F0F2FE680704BF23
:106DC000284670BD4FF0500080F31188BFF36F8FDD
:106DD000BFF34F8FFEE7000040F62440C2F20000F0
:106DE000016800291FBF01680A6D01320A65006849
:106DF0007047000046F64D1321F001014FF0807CF2
:106E0000C0F6000340E903316FF0020140F804CC02
:106E100040E9091244387047002808BF70472DE93F
:106E2000F0412DED048B4178827840F2D0244FF46C
:106E3000C066DFED910A9FED911ABFEE008AB7EEB2
:106E4000009AC2F20004F0EE481AB0EE492A62F34A
:106E50000A2100EE101AB8EEC00A84ED010A81780A
:106E6000C278C90862F34A1100EE101A4FF480612B
:106E7000B8EEC00A84ED020AC278037947799B0014
:106E800001EA872743EA92123A4300EE102AB8EE4D
:106E9000C00A84ED030A42798379520863F3CA1267
:106EA00000EE102AB8EEC00A84ED040A8279C37994
:106EB000120963F30A12A282C279037A477A5B004D
:106EC00006EA472743EAD2123A43E282427A837AB9
:106ED000920863F38A122283827AC37ADB0043EA40
:106EE00052126283027B437B63F30A22A283427BBA
:106EF000837BD20863F34A12E283827BC37B077CE5
:106F00009B0001EA872143EA921211432184017C0C
:106F1000407C490860F3CA11618494ED020AFEF7CF
:106F2000F3FFB1EE400ADFED560A9FED561AF0EE80
:106F3000481AB0EE492A84ED020A94ED010AFEF7E0
:106F4000E3FF84ED010ADFED500A9FED501AF0EEE9
:106F5000481AB0EE492A94ED030AFEF7D5FFB1EEC8
:106F6000400ADFED4B0A9FED4B1AF0EE481AB0EEE7
:106F7000492A84ED030A94ED040AFEF7C5FFB0EE3A
:106F8000408A84ED048A6068F9F776FA9FED320B47
:106F900006460F4658EC105B2A464346F9F7E7F9D8
:106FA00058B99FED2F0B3046394653EC102BF9F7AB
:106FB000F9F9002804BF00206060A068F9F75CFAC6
:106FC0002A46434606460F46F9F7D1F958B99FEDD0
:106FD000240B3046394653EC102BF9F7FEF9002804
:106FE00004BF0020A060E068F9F746FA9FED1E0B91
:106FF00006460F4653EC102BF9F7B9F958B99FED37
:107000001C0B3046394653EC102BF9F7E6F90028F3
:1070100004BF0020E06018EE100AF9F72DFA2A46A6
:10702000434606460F46F9F7A2F958B99FED0C0BF7
:107030003046394653EC102BF9F7CFF9002804BF3E
:107040000020206101202070BDEC048BBDE8F041E0
:10705000704700BF00BF00BF7B14AE47E17A84BF1A
:107060007B14AE47E17A843F9A9999999999A9BF7F
:107070009A9999999999A93F00007C4300E0CC44E2
:107080000000994300A0D3440000944200C0B144E2
:10709000000042430080C544D0E9013201699A6092
:1070A000826853604B68834208BF4A6000220261D5
:1070B00008680138086008687047000045F2DC6322
:1070C000C2F20003036045F2DC40C2F20000086037
:1070D000802010607047000045F63833C2F200038C
:1070E000036045F23870C2F2000008604FF480700F
:1070F0001060704700F108014FF0FF32C0E9011243
:10710000C0E9031100210160704700000021016106
:107110007047000080B5D1F800C01CF1010208D012
:1071200000F108029646DEF8042013686345F9D999
:1071300003E0D0F810E0DEF804204A609160C1F866
:1071400008E0CEF80410086101680131016080BDDB
:1071500042684A6093688B609368596091600861E7
:107160000168013101607047DFF80C00016841F4EB
:1071700070010160704700BF88ED00E04FF05000E3
:1071800080F31188BFF36F8FBFF34F8F40F29800E9
:10719000C2F2000001684A1C0029026000D070475A
:1071A0004EF60450CEF20000006810F0FF0F08BF4A
:1071B00070474FF0500080F31188BFF36F8FBFF31B
:1071C0004F8F00BFFEE7000040F29800C2F20000BF
:1071D000016839B10139016018BF7047002080F3A0
:1071E000118870474FF0500080F31188BFF36F8F04
:1071F000BFF34F8FFEE70000B0B50446002C08BF78
:10720000B0BD45F6943154F8040CA4F10805C2F25F
:1072100000010978002918BF4FF0004101420AD04F
:107220002A6892B14FF0500080F31188BFF36F8F3E
:10723000BFF34F8FFEE74FF0500080F31188BFF38C
:107240006F8FBFF34F8F00BFFEE7884344F8040CF5
:1072500000F042FB40F2202C54F8043CC2F2000C37
:10726000DCF804100CF114021944CCF8041000BF2F
:1072700011460A68AA42FBD34C680819A84202BF0B
:1072800023444B600D46E818904207D1DCF800001B
:1072900082421FBF5068184468601268A9422A6081
:1072A00018BF0D60DCF810000130CCF81000BDE80C
:1072B000B04001F075BC00004EF210000021CEF28B
:1072C00000000160816041F63F11C0F201014160A0
:1072D0000721016070470000EFF30580102814D3E8
:1072E0004EF2F031CEF20001405C40F23C21C2F29D
:1072F00000010978884208D24FF0500080F31188CD
:10730000BFF36F8FBFF34F8FFEE74EF60C5040F286
:107310003C21CEF20000C2F200010068496800F48E
:10732000E060884298BF70474FF0500080F31188AA
:10733000BFF36F8FBFF34F8FFEE7000045F6983C19
:10734000C2F2000CDCF80020FAB1634653F8082FB3
:10735000F2B1634653F8102FE2B1634653F8182F89
:10736000D2B1634653F8202FC2B1634653F8282F99
:10737000B2B1634653F8302FA2B1634653F8382FA9
:10738000002A18BF704707220DE0002263460AE07A
:10739000012208E0022206E0032204E0042202E0C7
:1073A000052200E0062219600CEBC201486070471C
:1073B00070B515460E460446FFF7E0FE94F844000B
:1073C000FF2804BF002084F8440094F84500FF28FB
:1073D00004BF002084F84500FFF7F6FEA06B28B933
:1073E00004F1240031462A4600F08EF92046BDE81B
:1073F0007040FFF7E3BB0000F0B581B00446C4B3B2
:1074000040F26015C2F20005286940B14FF050000B
:1074100080F31188BFF36F8FBFF34F8FFEE72869AA
:1074200040F62446C2F20006013028616F693068D8
:107430000430FFF731FE30683C44BC4244604FF0FA
:10744000010028BF0020002805D0E8693168043118
:10745000FFF760FE08E0A86931680431FFF75AFEC3
:10746000A86A844238BFAC6201F09AFB08B101B04F
:10747000F0BD4EF604504FF08051CEF20000016096
:10748000BFF34F8FBFF36F8F01B0F0BD88B1D1B1A3
:107490002DE9F04140F26014C2F200042269E2B129
:1074A0004FF0500080F31188BFF36F8FBFF34F8F01
:1074B000FEE74FF0500080F31188BFF36F8FBFF3EA
:1074C0004F8F00BFFEE74FF0500080F31188BFF3ED
:1074D0006F8FBFF34F8F00BFFEE722690132226139
:1074E000666902685518964202D2954202D320E09E
:1074F000954201D3B5421CD940F624480560C2F23A
:1075000000086769D8F800000430FFF7C5FDA81B24
:107510003D18D8F80000BD4245604FF0010028BF7B
:10752000002040B1E069D8F800100431FFF7F2FD07
:107530000BE0056009E0A069D8F800100431FFF7FE
:10754000E9FDA06A854238BFA56201F029FB002849
:10755000BDE8F04118BF70474EF604504FF080511F
:10756000CEF200000160BFF34F8FBFF36F8F704703
:10757000F0B581B00446FFF701FE002C02BF40F6D3
:107580002440C2F200000468251D2846FFF784FD50
:10759000A06A00281CBF04F11800FFF77DFD40F22F
:1075A000601640F62447C2F20006C2F200073068B7
:1075B000013030603868844217D0B0680138B0605C
:1075C00094F85900022808D0012803D068BB206B2A
:1075D000FFF712FE2046FFF70FFEB069006868B1A2
:1075E000B069C068C06840680AE006F13800294602
:1075F000FFF7AEFD70680130706002E04FF0FF30C1
:10760000B062FFF7E1FDF06810B13868844201D044
:1076100001B0F0BD306990B14FF0500080F3118897
:10762000BFF36F8FBFF34F8FFEE74FF0500080F333
:107630001188BFF36F8FBFF34F8F00BFFEE74EF689
:1076400004504FF08051CEF200000160BFF34F8F25
:10765000BFF36F8F01B0F0BD40F26011C2F20001C4
:107660004A6B0260496941607047000040F2601057
:107670000121C2F20000C16270470000F0B581B084
:107680000C4618B340F62446C2F2000631681831A1
:10769000FFF740FD40F26015C2F200056F693068E7
:1076A0000430FFF7F9FC601C19D030683C44BC4240
:1076B00044604FF0010028BF0020C8B1E86931687C
:1076C000043101B0BDE8F040FFF724BD4FF0500099
:1076D00080F31188BFF36F8FBFF34F8FFEE73168E0
:1076E00005F14C00043101B0BDE8F040FFF730BDBA
:1076F000A86931680431FFF70DFDA86A844238BFDC
:10770000AC6201B0F0BD00002DE9F04115460C4619
:1077100000B340F62447C2F2000739681831FFF77A
:1077200017FD40F26018C2F20008D8F814603868FB
:107730000430FFF7B1FC002D18BF4FF0FF3412D01A
:10774000601C10D1396808F14C000431BDE8F041EB
:10775000FFF7FEBC4FF0500080F31188BFF36F8F2E
:10776000BFF34F8FFEE738683444B44244604FF0B3
:10777000010028BF002038B1D8F81C003968043156
:10778000BDE8F041FFF7C6BCD8F8180039680431ED
:10779000FFF7C0FCD8F82800844238BFC8F828405A
:1077A000BDE8F08170B5044624B3226D1AB3E06CD5
:1077B000884238BF0846012A1CD1E16A814208BFCD
:1077C00070BD40F62442C2F200021268A2421CD0F0
:1077D000E06240F62846A269C2F20006002AA4BF71
:1077E000C0F13800A06101EB8100616906EB800007
:1077F000814214D070BD4FF0500080F31188BFF368
:107800006F8FBFF34F8F00BFFEE74FF0500080F344
:107810001188BFF36F8FBFF34F8F00BFFEE7251DA9
:107820002846FFF739FC40F26011E06AC2F200011D
:107830000A6A904288BF086200EB8000294606EB86
:107840008000BDE87040FFF783BC000010B586B033
:10785000002405A804A903AACDE90444FFF72EFCDF
:10786000DDE9032005990023CDE9004046F2E570EB
:10787000029117A1C0F6000000F012FF40F2601460
:107880000028C2F20004606216D001F003FA411C25
:1078900014D0012810D14FF0500080F31188BFF3AD
:1078A0006F8FBFF34F8F4FF0FF30A0620120E06079
:1078B0000020606100F05EF806B010BD4FF050008F
:1078C00080F31188BFF36F8FBFF34F8FFEE700BFC8
:1078D00049444C450000000040F26010C2F2000034
:1078E000016901310161704780B540F2601EC2F24A
:1078F000000EDEF8101000291EBF0121CEF82C105A
:1079000080BD002140F6284CCEF82C10C2F2000CAD
:10791000DEF8201001EB81035CF8232052B90CEB58
:107920008302A2F1140300BFD1B153F81429013925
:10793000002AF9D001EB81020CEB820353F8042FEB
:107940005268181D1A60824204BF52681A60D068DB
:1079500040F62442C2F200021060CEF8201080BD32
:107960004FF0500080F31188BFF36F8FBFF34F8F3C
:10797000FEE700004EF200404CF27021CEF2000013
:10798000C4F20F11D0F800294B1C9A4209D14FF0D4
:10799000500080F31188BFF36F8FBFF34F8F00BF8C
:1079A000FEE7D0F800298A4209D14FF0500080F359
:1079B0001188BFF36F8FBFF34F8F00BFFEE7B0B5E5
:1079C00084B001780291FF21017001788DF80710D1
:1079D0009DF8071001F0500240F23C21C2F2000174
:1079E0000A7007224A609DF90720B2F1FF3F49DC87
:1079F000062200BF4A60013A9DF807305B008DF80F
:107A000007309DF90730002BF4DB022A3AD14FF4FE
:107A100040724A6002990170D0F8201941F4700157
:107A2000C0F82019D0F8201941F07041C0F8201991
:107A3000FFF742FC40F298040025C2F200042560E2
:107A4000FFF792FB4EF63470CEF20000016841F071
:107A500040410160FEF70CFFFFF746FF03952068E9
:107A60004FF0500181F31188BFF36F8FBFF34F8F39
:107A7000013001D0FEE700BF03980028FCD00020B1
:107A800004B0B0BD4FF0500080F31188BFF36F8F8A
:107A9000BFF34F8FFEE7000080B54FF0500080F33A
:107AA0001188BFF36F8FBFF34F8F00F099FE00284E
:107AB0001FBF4EF60450CEF200004FF0805101601F
:107AC000002080F3118880BD70B505465020FFF777
:107AD000B3F8044674B30026012084F8466024609D
:107AE000C4E90F06FFF74AFB2068D4E90F1202FB36
:107AF00001030139A360A663606001FB0200E0603E
:107B0000FF2084F8440084F8450004F11000FFF7DA
:107B1000F1FA04F12400FFF7EDFAFFF755FB2046D8
:107B200000210022002384F84C502660C4E902663C
:107B300000F00AF9204670BD70B582B00C460546CB
:107B4000BCB350200190019850283CD101980026E8
:107B5000012084F846002460C4E90F06FFF70EFBFD
:107B60002068D4E90F1202FB01030139A360A66368
:107B7000606001FB0200E060FF2084F8440084F8AC
:107B8000450004F11000FFF7B5FA04F12400FFF7F7
:107B9000B1FAFFF719FB204600210022002384F8E8
:107BA0004C502660C4E9026600F0CEF8204602B0D0
:107BB00070BD4FF0500080F31188BFF36F8FBFF39B
:107BC0004F8F00BFFEE74FF0500080F31188BFF3E6
:107BD0006F8FBFF34F8F00BFFEE700002DE9F0412C
:107BE000074614460E46A7B306FB07F05030FFF7D2
:107BF00023F8054655B34FF00008002E284685F8B7
:107C0000468018BF50302860C5E90F76FFF7B6FAF6
:107C10002868D5E90F1202FB01030139AB60C5F8F2
:107C20003880686001FB0200E860FF2085F84400AE
:107C300085F8450005F11000FFF75CFA05F1240016
:107C4000FFF758FAFFF7C0FA85F84C402846BDE820
:107C5000F0814FF0500080F31188BFF36F8FBFF3B6
:107C60004F8F00BFFEE70000B0B582B01C4660B188
:107C7000ACB1F1B9EAB14FF0500080F31188BFF315
:107C80006F8FBFF34F8F00BFFEE74FF0500080F3C0
:107C90001188BFF36F8FBFF34F8F00BFFEE74FF028
:107CA000500080F31188BFF36F8FBFF34F8F00BF79
:107CB000FEE751B14AB94FF0500080F31188BFF38D
:107CC0006F8FBFF34F8F00BFFEE75023069D0193D8
:107CD000019B502B2DD1019B00294FF0010384F80B
:107CE000463008BF22462260C4E90F01FFF746FA7A
:107CF0002068D4E90F1202FB01030139A3600023BD
:107D0000A363606001FB0200E060FF2084F8440090
:107D100084F8450004F11000FFF7ECF904F12400A9
:107D2000FFF7E8F9FFF750FA84F84C50204602B00C
:107D3000B0BD4FF0500080F31188BFF36F8FBFF3D9
:107D40004F8F00BFFEE700002DE9F04F83B00446DF
:107D500017461D460E46002C029714D0EEB1022D98
:107D600003D1E06B012840F0A38000F019FD00BBB7
:107D7000FFB14FF0500080F31188BFF36F8FBFF356
:107D80004F8F00BFFEE74FF0500080F31188BFF324
:107D90006F8FBFF34F8F00BFFEE7206C0028DED04F
:107DA0004FF0500080F31188BFF36F8FBFF34F8FF8
:107DB000FEE7FFF7E3F9A06B022D5AD0E16B884292
:107DC00057D304F110086F464FF0000A02980028BC
:107DD00000F07F80BAF1000F04D13846FFF73CFC79
:107DE0004FF0010AFFF7F0F9FFF776FDFFF7C6F94C
:107DF00094F84400FF2804BF002084F8440094F85D
:107E00004500FF2804BF002084F84500FFF7DCF997
:107E1000384602A900F092FB00285DD1FFF7AEF9C9
:107E2000D4F838B0D4F83C90FFF7CEF9CB4515D153
:107E300002994046FFF722FC2046FEF7BFFE00F005
:107E4000AFFE80B94EF604504FF08051CEF20000E4
:107E50000160BFF34F8FBFF36F8F04E02046FEF742
:107E6000ADFE00F09DFEFFF789F9A06BE16B884243
:107E7000ACD2A76B226C22B3BDB3E0683146F8F7F1
:107E8000E3F9E168206C091AE160226891423FBF82
:107E90004042A1680844E060002FA5F10201384685
:107EA000B1FA81F118BF0120490908403F1A29E0C1
:107EB0004FF0500080F31188BFF36F8FBFF34F8FE7
:107EC000FEE720680025E8B9A06800F091FDA560F4
:107ED00019E0FFF779F904E02046FEF76FFE00F0A5
:107EE0005FFE002003B0BDE8F08F60683146F8F710
:107EF000ABF96068216C08446060A168884224BFC7
:107F0000206860600020791CA16354F8241F79B1B7
:107F1000204600F003FEB8B14EF604514FF08050F9
:107F2000CEF200010860BFF34F8FBFF36F8F0BE0FD
:107F300050B14EF604514FF08050CEF2000108606F
:107F4000BFF34F8FBFF36F8FFFF73EF9012003B0F0
:107F5000BDE8F08F2DE9F04705461E4614460F4652
:107F6000E5B127B3022E02D1E86B012852D1FFF709
:107F7000B3F9EFF311884FF0500080F31188BFF38D
:107F80006F8FBFF34F8F022EA86B1CD0E96B884216
:107F900019D388F311880020BDE8F0874FF0500016
:107FA00080F31188BFF36F8FBFF34F8FFEE7286C0C
:107FB0000028D7D04FF0500080F31188BFF36F8FA7
:107FC000BFF34F8FFEE795F84590A86BD5F838A022
:107FD0002A6C002A27D0002E2DD0E8683946F8F701
:107FE00033F9E968286C091AE9602A6891423FBFB1
:107FF0004042A9680844E860BAF1000FA6F1020106
:108000005046B1FA81F118BF012049090840AAEB96
:10801000000A1DE04FF0500080F31188BFF36F8F0E
:10802000BFF34F8FFEE7286890B9A86800F0E0FC26
:108030000020A8600CE068683946F8F705F9686820
:10804000296C08446860A968884224BF2868686071
:108050000AF10100B9F1FF0FA86308D009F101008E
:1080600085F84500012088F31188BDE8F08755F8B0
:10807000240F78B1284600F051FD0146002C4FF046
:10808000010018BF0029EED00120206088F311887C
:10809000BDE8F08788F311880120BDE8F087000073
:1080A000B0B50446A4B1A56800F074FB85421CBFBE
:1080B0000020B0BDE0680138E0601CBF0120B0BD09
:1080C0002046002100220023FFF73EFE0120B0BD24
:1080D0004FF0500080F31188BFF36F8FBFF34F8FC5
:1080E000FEE700002DE9F04F85B0044616460D4628
:1080F000002C04960FD0002D46D000F051FBA0B903
:108100009EB14FF0500080F31188BFF36F8FBFF323
:108110004F8F00BFFEE74FF0500080F31188BFF390
:108120006F8FBFF34F8F00BFFEE7FFF727F8D4F83C
:108130003890B9F1000F34D0226C52B1E068811848
:10814000E160A0688142284624BF2168E160F8F719
:108150007BF8A9F10100A06354F8100F70B120461C
:1081600000F0DCFC50B14EF604514FF08050CEF2DE
:1081700000010860BFF34F8FBFF36F8FFFF724F844
:10818000012005B0BDE8F08F206C0028B5D04FF07D
:10819000500080F31188BFF36F8FBFF34F8F00BF84
:1081A000FEE7002E65D004F124004FF0000A02AF74
:1081B0000DF110084FF0000B019000BFBBF1000F54
:1081C00004D13846FFF748FA4FF0010BFEF7FCFFE9
:1081D000FFF782FBFEF7D2FF94F84400FF2808BFA8
:1081E00084F844A094F84500FF2808BF84F845A00F
:1081F000FEF7EAFF3846414600F0A0F960B120469C
:10820000FEF7DCFC00F0CCFCFEF7B8FFA66BFEF737
:10821000DBFF1EBB2FE000BFFEF7B0FFA66BFEF733
:10822000D3FF2EB12046FEF7C9FC00F0B9FC15E0E3
:1082300004990198FFF722FA2046FEF7BFFC00F0F0
:10824000AFFC58B94EF604504FF08051CEF200000A
:108250000160BFF34F8FBFF36F8F00BFFEF78EFF3C
:10826000D4F83890B9F1000F7FF466AF0498002875
:10827000A4D1FEF7A9FF002005B0BDE8F08F0000F3
:108280002DE9F04381B0054691460E4635B376B3ED
:10829000FFF722F8EFF311884FF0500080F31188B8
:1082A000BFF36F8FBFF34F8FAC6B64B395F844701F
:1082B0002A6C52B1E8688118E960A86881423046AA
:1082C00024BF2968E960F7F7BFFF601EFF2FA8638E
:1082D0001BD0781C85F84400012028E04FF05000A6
:1082E00080F31188BFF36F8FBFF34F8FFEE7286CC9
:1082F0000028CDD04FF0500080F31188BFF36F8F6E
:10830000BFF34F8FFEE7002011E055F8100F68B162
:10831000284600F003FC01460120B9F1000F06D009
:1083200000291CBF0120C9F8000000E0012088F3EB
:10833000118801B0BDE8F0832DE9F04F85B0044607
:108340000D46002C04950AD0206C90B14FF05000DF
:1083500080F31188BFF36F8FBFF34F8FFEE74FF0AD
:10836000500080F31188BFF36F8FBFF34F8F00BFB2
:10837000FEE700F015FA50B94DB14FF0500080F310
:108380001188BFF36F8FBFF34F8F00BFFEE7FEF77B
:10839000F5FEA06BF0B10138A063206810B9FEF7BC
:1083A0001BFDA06054F8100F70B1204600F0B6FB22
:1083B00050B14EF604514FF08050CEF200010860EB
:1083C000BFF34F8FBFF36F8FFEF7FEFE012005B0A6
:1083D000BDE8F08F04F124004FF0000902AE04AFB5
:1083E0004FF0000B4FF0000A019061E0BBF1000F6D
:1083F00004D13046FFF730F94FF0010BFEF7E4FEF1
:10840000FFF76AFAFEF7BAFE94F84400FF2808BFA7
:1084100084F8449094F84500FF2808BF84F84590FC
:10842000FEF7D2FE3046394600F088F860B12046AB
:10843000FEF7C4FB00F0B4FBFEF7A0FEA56BFEF751
:10844000C3FE7DB943E000BFFEF798FED4F8388044
:10845000FEF7BAFEB8F1000F09D02046FEF7AEFBDA
:1084600000F09EFBFEF78AFEA06B08B393E720683E
:1084700038B9FEF783FEA06800F006FB8246FEF7DF
:10848000A3FE04990198FFF7F9F82046FEF796FB42
:1084900000F086FB0028E5D14EF604504FF08051E5
:1084A000CEF200000160BFF34F8FBFF36F8FD9E7AB
:1084B000049800289AD1BAF1000F18D04FF050005C
:1084C00080F31188BFF36F8FBFF34F8FFEE7BAF1D0
:1084D000000F0ED0FEF752FE606A20B1206B0068DC
:1084E000C0F1380100E00021A068FFF75BF9FEF75A
:1084F0006BFE002005B0BDE8F08F000070B50446AB
:108500000D466CB1A66800F045F9864211D02046B0
:108510002946FFF711FF002804BF002070BD09E0C5
:108520004FF0500080F31188BFF36F8FBFF34F8F70
:10853000FEE70120E1680131E16070BDB0B504469D
:108540000D46ACB1EDB1FEF719FE40F2601CC2F26F
:10855000000CDCF8142029684B1C1CD0D4E9000E58
:10856000DCF83430834218D0724516D3012425E05C
:108570004FF0500080F31188BFF36F8FBFF34F8F20
:10858000FEE74FF0500080F31188BFF36F8FBFF309
:108590004F8F00BFFEE7002410E0A2EB0E029142D5
:1085A00009D9881A2860DCF834002060DCF814004F
:1085B0006060002402E0002001242860FEF704FE31
:1085C0002046B0BD2DE9F04F81B0904682469946D5
:1085D0000F464FEA88052846FEF72EFB04465CB39B
:1085E0005C20FEF729FB06461EB3DDF828B000200C
:1085F00034632946A52286F859002046F7F736FE4F
:10860000306B002F00EB8800A0F1040020F0070879
:1086100017D006F1340000217A5C42544A1C0F2A1C
:1086200003D8795C00291146F6D1002086F8430072
:108630000AE02046FEF7E0FD4FF0FF3001B0BDE854
:10864000F08F002086F83400BBF1370F06F10400EC
:108650004FF0000428BF4FF0370BC6F82CB0C6E926
:1086600013B4FEF753FD06F11800FEF74FFDCBF1F2
:108670003800366151464A46B061404676627465BC
:1086800086F85840FEF7B6FB30600B98002818BFFC
:1086900006603046FDF756FF012001B0BDE8F08FBF
:1086A0002DE9F04782B08246DDE90B049946154674
:1086B0000F4640B38CB35C21019101995C2936D1FE
:1086C00001990A9E2063A522022184F85910A9006D
:1086D000F7F7CCFD206B002F00EB8500A0F1040024
:1086E00020F007082DD004F1340000217A5C4254B8
:1086F0004A1C0F2A03D8795C00291146F6D10020C4
:1087000084F8430020E04FF0500080F31188BFF35D
:108710006F8FBFF34F8F00BFFEE74FF0500080F325
:108720001188BFF36F8FBFF34F8F00BFFEE74FF08D
:10873000500080F31188BFF36F8FBFF34F8F00BFDE
:10874000FEE7002084F83400372E04F104004FF0D7
:10875000000528BF3726E662C4E91365FEF7D6FC9C
:1087600004F11800FEF7D2FCC6F13800246151462E
:108770004A46A06140466462656584F85850FEF739
:1087800039FB20602046FDF7DDFE204602B0BDE843
:10879000F087000040F62440C2F2000000687047F5
:1087A00040F26010C2F20000C168002904BF01203D
:1087B000704701690020002908BF022070470000AF
:1087C00040F26010C2F200004069704780B5FEF7C9
:1087D00083FD40F26010C2F20000406980BD0000DD
:1087E0002DE9F04740F26016C2F20006306930B160
:1087F000306B0024013030632046BDE8F08770699B
:1088000010F1010AC6F814A03ED0B06A824501D228
:1088100000244AE0B0690068002842D040F62848A9
:1088200040F624490024C2F20008C2F2000900BF49
:10883000B069C068C7683D4655F8040F824533D318
:108840002846FEF729FCB86A00281CBF07F118006B
:10885000FEF722FCF86A316A8842294688BF3062F6
:1088600000EB800008EB8000FEF772FCF86AD9F894
:108870000010C96A884228BF0124B0690068002836
:10888000D6D14FF0FF300FE0B069006828B34FF049
:10889000500080F31188BFF36F8FBFF34F8F00BF7D
:1088A000FEE74FF0FF300024B06240F6244040F66F
:1088B0002841C2F20000C2F200010068C06A00EB69
:1088C000800051F82000012888BF0124F06A0028A8
:1088D00018BF01242046BDE8F087B069F169B16195
:1088E000F061706B01307063B069006820B1B069ED
:1088F000C068C068406801E04FF0FF30B06284E7B4
:108900002DE9F04381B01E46154688460746FEF71E
:1089100035FC40F62444C2F20004206890F8580068
:10892000022845D02068002E416D21EA07014165EB
:108930004FF00101206880F8581039D040F26019DA
:10894000C2F20009D9F8147020680430FEF7A4FBC5
:10895000701C0FD020683E44BE4246604FF00100BC
:1089600028BF002068B1D9F81C0021680431FEF747
:10897000D1FB12E0216809F14C000431FEF7E8FB5D
:108980000BE0D9F8180021680431FEF7C3FBD9F8D1
:108990002800864238BFC9F828604EF604504FF0D0
:1089A0008051CEF200000160BFF34F8FBFF36F8F95
:1089B000FEF70AFCFEF7E2FB002D1EBF2068406DAB
:1089C00028600025206890F858100020022905D161
:1089D000216801254A6D22EA08024A65216881F86A
:1089E0005800FEF7F1FB284601B0BDE8F083000017
:1089F000B0B50446002C04BF0020B0BD40F62440B2
:108A0000C2F200000068A04209D04FF0500080F38D
:108A10001188BFF36F8FBFF34F8F00BFFEE7206D4C
:108A200038B3013820654FF0000018BFB0BDE16ACF
:108A3000E26C91421CD0251D2846FEF72DFBE06C10
:108A4000C0F13801E062A16140F26011C2F20001A0
:108A50000A6A904288BF086240F6284100EB800015
:108A6000C2F2000101EB80002946FEF771FB0120F4
:108A7000B0BD4FF0500080F31188BFF36F8FBFF38C
:108A80004F8F00BFFEE70000F0B581B00446002C18
:108A900002BF002001B0F0BD40F62446E06AC2F2F9
:108AA00000063168C96A884216D2A16940F6284793
:108AB00000EB8000C2F2000707EB80000029A1BF95
:108AC0003168C96AC1F13801A161616981420CD084
:108AD0003068C06AE0621EE0E16C3068C26A002063
:108AE000914238BF012001B0F0BD251D2846FEF798
:108AF000D3FA306840F26011C2F20001C06AE0624D
:108B00000A6A904288BF086200EB8000294607EBA2
:108B10008000FEF71DFB012001B0F0BD70B5C068FC
:108B2000C5688DB105F118042046FEF7B5FA40F28C
:108B30006016C2F20006306978B106F16000214685
:108B4000FEF706FB2C351DE04FF0500080F3118836
:108B5000BFF36F8FBFF34F8FFEE72C1D2046FEF74C
:108B60009BFA55F82C0F316A884240F6284188BF9D
:108B7000306200EB8000C2F2000101EB8000214670
:108B8000FEF7E6FA40F624412868C2F200010968BF
:108B9000C96A884292BF00200120F06270BD0000C7
:108BA0002DE9F04381B040F26015C2F2000528695A
:108BB00068B1FEF7E3FA286901382861286980B1B5
:108BC0000024FEF701FB204601B0BDE8F0834FF022
:108BD000500080F31188BFF36F8FBFF34F8F00BF3A
:108BE000FEE7A868A0B3286EB8B340F6284940F65F
:108BF00024474FF00108C2F20009C2F2000700BF8B
:108C0000E86EC66806F11800FEF746FA341D2046E5
:108C1000FEF742FAF06A296A8842214688BF286234
:108C200000EB800009EB8000FEF792FAF06A3968E9
:108C3000C96A884228BFC5F82C80286E0028DFD179
:108C4000A869006830B1A869C068C068406803E0DE
:108C50000024B6E74FF0FF30A8622C6B4CB1012620
:108C6000FFF7BEFD002818BFEE62013CF8D10020DE
:108C70002863E86A60B14EF604504FF08051012439
:108C8000CEF200000160BFF34F8FBFF36F8F98E704
:108C9000002496E770B586B0FEF770FA40F2E01651
:108CA000C2F20006306810BB06F114042046FEF73D
:108CB00021FA06F128052846FEF71CFA40F6843210
:108CC00040F2F04300201021C6E902450090C2F2B4
:108CD0000002C2F200030A20FEF7C6FF002830603F
:108CE00005D049F2B441C0F60001FEF727FBFEF7BC
:108CF0006BFA3068E0B1002004A903AACDE90400B2
:108D000005A8FEF7E9F9DDE9032005990223CDE97D
:108D1000003046F6811002910AA10023C0F600003F
:108D2000FFF7BEFC002870601EBF012006B070BDBA
:108D30004FF0500080F31188BFF36F8FBFF34F8F58
:108D4000FEE700BF546D72205376630041000802B5
:108D500018BF04200A0E18BF40F001004FF07F42F8
:108D600032EA010108BF40F00200012808BF0520D7
:108D7000704710EE100A20F0004000EE100A704715
:108D800010EE101A08B5444A6846B2EB410F28D9D4
:108D90004FF0E640B0EB410F94BF00204FF0FF30A2
:108DA00000900098002861DB60EE000A10F0010FCF
:108DB00045D010F0020FDFED391A9FED391A00EEA1
:108DC000A11ADFED381A40EE811A21EEA01AF0EE5A
:108DD000400A40EE010A08BFF1EE600AB0EE600AF8
:108DE00008BD314B21F0004293423CD911F0004FB5
:108DF000DFED2E0A20EE201ADFED2D0A19BF31EE2D
:108E0000601A71EE200A31EE201A71EE600ABDEE92
:108E1000E01A11EE100A9FED271A00F0030000EE91
:108E2000C10A9FED251A009000EEC10A9FED231A9A
:108E300000EEC10A9FED221A00EEC10AB1E79FEDD4
:108E4000211A9FED210A10F0020F00EE810A9FED1A
:108E50001F1A00EE801AB7EE000A00EE810A18BF52
:108E6000B1EE400A08BD00F0F1F99AE710EE100AE1
:108E70004000B0F17F4F3CBFB7EE000A08BD07D1FC
:108E80004FF0010000F09CFABDE8084000F0CEB9B8
:108E9000BDE8084000F0C6B9B61F927E336D4CB9EC
:108EA000DA82083CA0AA2ABE490E494683F9223F2D
:108EB0000000004B0000C93F00A0FD390020A23394
:108EC0001A61342CB93AB2BACA9F2A3DDDFFFFBEFF
:108ED00010B52DED028BB0EE608AF0EE408A18EEF0
:108EE000101A18EE900AF7F78DFB00F07040B0F101
:108EF000005F0CD018EE100A20F00040C0F1FF40D7
:108F0000C00F02BFB0EE480ABDEC028B10BDB0EE40
:108F1000680ABDEC028B10BD00B510EE101A2DEDE5
:108F2000028B81B0524A6846B2EB410F2ED94FF006
:108F3000E640B0EB410F94BF00204FF0FF300090AF
:108F40000098B0EE408A00286ADB10F0010F4BD089
:108F500068EE080A9FED471A9FED470A00EE810A66
:108F60009FED461A10F0020F00EE801AB7EE000ACD
:108F700000EE810A02BF01B0BDEC028B00BD00BF54
:108F800001B0B1EE400ABDEC028B00BD3C4B21F0BC
:108F90000042934241D911F0004FDFED3A0A20EE32
:108FA000201ADFED390A19BF31EE601A71EE200A7E
:108FB00031EE201A71EE600ABDEEE01A11EE100AD1
:108FC0009FED321A00F0030000EEC10A9FED301A47
:108FD000009000EEC10A9FED2F1A00EEC10A9FED2E
:108FE0002E1A00EEC10AABE728EE080A9FED2B1AF5
:108FF000DFED2B0A10F0020F40EE010A9FED291A57
:1090000000EE201A61EE000AB0EE480A08EE200ACF
:10901000B6D101B0BDEC028B00BD00F017F98FE7AF
:1090200018EE100A4000B0F17F4F0DD218EE100A72
:10903000FFF78CFE042808BF00F000F9B0EE480AE4
:1090400001B0BDEC028B00BD09D1012000F0B8F9E0
:1090500001B0BDEC028B5DF804EB00F0E7B801B0A5
:10906000B0EE480ABDEC028B5DF804EB00F0DAB814
:10907000B61F927EB93AB2BACA9F2A3DDDFFFFBE43
:10908000490E494683F9223F0000004B0000C93FCA
:1090900000A0FD390020A2331A61342C336D4CB985
:1090A000DA82083CA0AA2ABE00B510EE101A2DEDF7
:1090B000028B81B04D4A6846B2EB410F3CD94FF06C
:1090C000E640B0EB410F94BF00204FF0FF3000901E
:1090D0000098B0EE408A00285FDB28EE080ADFED3A
:1090E000440A9FED441A00EE201ADFED430A40EED9
:1090F000010A9FED421A00EE201ADFED410A10F03E
:10910000010F40EE010A9FED3F1A00EE201A61EEBA
:10911000000AB0EE480A08EE200A02BF01B0BDEC1A
:10912000028B00BDBFEE001A01B0C1EE000ABDEC1B
:10913000028BB0EE600A00BD334B21F00042934237
:1091400028D911F0004FDFED310A20EE201ADFEDB3
:10915000300A19BF31EE601A71EE200A31EE201A82
:1091600071EE600ABDEEE01A11EE100A9FED291AA9
:1091700000F0030000EEC10A9FED271A009000EEF8
:10918000C10A9FED261A00EEC10A9FED251A00EED6
:10919000C10A9DE700F05AF89AE718EE100A40005D
:1091A000B0F17F4F0DD218EE100AFFF7CFFD042863
:1091B00008BF00F043F8B0EE480A01B0BDEC028BE6
:1091C00000BD09D1012000F0FBF801B0BDEC028B1D
:1091D0005DF804EB00F02AB801B0B0EE480ABDEC2F
:1091E000028B5DF804EB00F01DB80000B61F927E04
:1091F000BCE9223C0B6D063B8A76CE3CACB5593DB2
:1092000035A1083E29AAAA3E490E494683F9223FC4
:109210000000004B0000C93F00A0FD390020A23330
:109220001A61342C30EE000A70470000DFED020AAC
:1092300080EEA00A70470000000000009FED020AC7
:1092400020EE000A70470000000000102DE9F00138
:109250004FF07F42B2EB410F9FBF4FF0FF310160F3
:10926000BDE8F00170474FF0004242EA0123C1F32C
:10927000C752783A551112F01F0C434CCCF120061E
:109280007C44C1F3C752A2F178024FEA621204EBA8
:10929000820254F8254008BFD2E9015612D0556821
:1092A00004FA0CF425FA06F73C43976805FA0CF526
:1092B00027FA06F8D26807FA0CFCF24045EA0805DE
:1092C0004CEA0206A4FB034CA5FB0352A6FB036376
:1092D0001D449D4234BF012600261319334416B1A4
:1092E000934202D903E0934201D2012200E000221E
:1092F000624402F1200C9206DC0C42EA443200EE99
:10930000102A5B03DFED210AF8EEC01A00EE103AD6
:109310004FEA9C1C11F0004FB8EE400AC0F800C0A4
:1093200020EE201A00EE105ADFED190AB8EE400ABE
:1093300020EE200A71EE810A70EE800A10EE902A6B
:1093400002F500626FF30B0200EE902A70EEE11A54
:1093500031EEC11ADFED101A30EE411A9FED0D0A01
:1093600020EE800A01EE210A9FED0C1A00EE810A20
:1093700004BFBDE8F0017047CCF180510160BDE849
:10938000F001B1EE400A70474801000000000036CD
:109390000000802C22AAFD29DB0FC92F0000C92F55
:1093A00002E008C8121F08C1002AFAD170477047AE
:1093B000002001E001C1121F002AFBD1704700000C
:1093C0000149086070470000040000200000000010
:1093D0006E83F9A22915444ED15727FCC0DD34F520
:1093E000999562DB4190433CAB6351FE00401C46C3
:1093F000000080460060EA46000000000000000017
:10940000010203040607080900000000010203042A
:10941000C3940008000000000000000000000000ED
:109420000000000000040000300000000000000008
:1094300000000000CD9400080000000000000000C3
:109440000000000000000000000400001800000000
:109450000000000000000000B994000800000000B7
:1094600000000000000000000000000000040000F8
:1094700018000000000000000000000000061016A8
:1094800000061016A894000800000000000000006C
:1094900000000000000000000002000018000000B2
:1094A000000000000000000064656661756C745483
:1094B00061736B00546D72510079616F6B6F6E67F1
:1094C0007169005461736B5F496E697400746573F0
:1094D000740000000095000800000020A0000000BB
:1094E000A0930008A0950008A0000020385F0000AD
:1094F000B093000800000000000000000000000021
:10950000000000000000000001000000100000004A
:10951000000000000024F40000000102010001002E
:10952000000002020100010000000302010001002E
:1095300000000402010001006F12833A0000803F26
:1095400000000000000000000000803F0000803F9D
:10955000000080BF000080BF0000003F0000803F8F
:1095600000000000000000000000803F0000803F7D
:10957000000080BFDB0FC94000000000000048422F
:109580000000484201000000000040400000404050
:109590000000004000007A46AAAAAAAA0000000023
:040000050800018965
:00000001FF
